:1080000000000120C903010045DB000045DB000042
:1080100045DB000045DB000045DB00000000000000
:1080200000000000000000000000000045DB000030
:1080300045DB00000000000045DB00001D8600005D
:1080400045DB000045DB000045DB000045DB0000B0
:1080500045DB000045DB000045DB000045DB0000A0
:1080600045DB000045DB000045DB000045DB000090
:1080700045DB000045DB000045DB000045DB000080
:1080800045DB000045DB000045DB000045DB000070
:1080900045DB000045DB000045DB000045DB000060
:1080A00045DB000061CD000045DB000045DB000042
:1080B00045DB000045DB000045DB000045DB000040
:1080C00045DB000045DB000045DB000045DB000030
:1080D00045DB000045DB000045DB000075C9000002
:1080E00045DB000045DB000045DB000045DB000010
:1080F00045DB000045DB000045DB000045DB000000
:1081000045DB000045DB000045DB000045DB0000EF
:1081100045DB000061ED000045DB000045DB0000B1
:1081200045DB000045DB000045DB000045DB0000CF
:1081300045DB000045DB000045DB000045DB0000BF
:1081400045DB000045DB00007187000045DB0000D7
:1081500045DB000045DB000045DB000045DB00009F
:1081600045DB0000B1C9000045DB000045DB000035
:1081700045DB000045DB000045DB000045DB00007F
:0881800045DB000045DB0000B7
:10840000FFFFFFFFFFFFFFFFFFFFFFFF7EF9FFFF03
:1084100010B5054C237833B9044B13B10448AFF3BE
:1084200000800123237010BD0086FF1F00000000A4
:10843000A40B01000C4B43B10C480D4910B5AFF330
:1084400000800C48036823B910BD0A48036833B99B
:108450007047094B002BF7D0BDE810401847064B7A
:10846000002BF5D0184700BF00000000A40B01004E
:108470000486FF1F6C85FF1F0000000080F3118839
:1084800070472F4B41F238015A5842F478525A50F3
:108490002C4A927902F00C020C2A4FD041F244028D
:1084A0002949995003F558339A78110748BF9A78AB
:1084B000264944BF42F008029A70214B41F244021F
:1084C000995041F204015A5842F4803242F0C002FD
:1084D0005A501A6842F440221A6003F5E833242205
:1084E0005A701B4A80211170A2221A70DA7802F0A9
:1084F0001F02DA7003221A7100225A719A799207C8
:10850000FCD59A79D006FCD40E4B19469A7902F024
:108510000C02082AFAD140225A718B7903F00C031D
:10852000082BFAD1074B1A4699794906FCD5222126
:108530001970937903F00C030C2BFAD1704700BF2C
:1085400000700440004006400000330100001301A9
:10855000005006402B4B5A7902F0E0025A711A790A
:1085600002F0F8021A71284A136843F004031360FA
:10857000264A136823F0784323F001031360244B49
:108580001A7802F08C0242F050021A705A7802F007
:108590009C0242F040025A709A7802F0E6029A7009
:1085A0001C4A0023137083F311881B4B012283F8AC
:1085B000182383F81923022283F83C2383F83D23F0
:1085C00083F84B2383F84C2383F84D2383F84E2301
:1085D00083F84F23032283F81F2383F8212383F892
:1085E000232383F8252383F84223042283F82723B7
:1085F000052283F84923062283F83B23072283F8C8
:108600003523704700F007404080044000D0004010
:1086100000D0074000E0074000E100E00C4A13688A
:10862000013313600B4A1368013313600A4B1A6855
:108630003AB11A68013A1A601B6813B9074B012254
:108640001A70074B1A6812B11A68013A1A6070471B
:108650001C86FF1FF095FF1F2493FF1F2093FF1F11
:108660002893FF1F024B034A5A6007221A60704783
:1086700010E000E000770100014B1868704700BF70
:108680001C86FF1F1449154B41F22802072888BF9A
:10869000002010B553F82030114CB4FBF3F48B5884
:1086A00043F480638B500F4B4FF440729A63422027
:1086B000DA6305F065FA0C4B0022DA709A709A7151
:1086C000DA725A71C4F30422E4B21A705C70DA7878
:1086D00042F02C02DA7010BD0070044068090100FD
:1086E000C0C62D0000B0044000A00E40094A136827
:1086F00051680133202B08BF00238B4208D011683A
:10870000114408721360044AD37843F08003D37095
:10871000704700BF2086FF1F00A00E400A4B996AD9
:10872000DA6A91420DD09A6A511C1A44996292F801
:10873000302002709A6A202A01D100229A62012018
:1087400070470020704700BF2086FF1F044B1A7837
:1087500002F0FF0012B100221A700120704700BF22
:108760002093FF1F014B1865704700BF2086FF1F35
:1087700030B526480179C9B28C0617D5244BDA6A80
:108780009C6A0132202A08BF0022A2421BBFDC6A79
:10879000C579C27918191EBFEDB280F83050DA627F
:1087A0001C4A052010601A6D1B4B1A604A0608D53A
:1087B0001A4B4FF480529A60144AD37803F0BF03E7
:1087C000D3700B061BD5144B1868C0B9104B196831
:1087D0005A68914214D0114A4FF4805151605A683E
:1087E000511C1A445960117A084AC9B2D1715968AA
:1087F000202908BF5860D37843F04003D37030BDC0
:10880000024AD37803F07F03F8E700BF00A00E40D0
:108810002086FF1F2493FF1F2893FF1F80F00F4027
:1088200062B67047FFF7FCBF72B67047FFF7FCBF38
:108830004FF0E02318B1034AC3F80C2D7047024AE9
:10884000FAE700BF0400FA050100FA05F7B544484D
:10885000444C454D454E4FF480731622436083606F
:108860000361A2601E226261414A53629364D36431
:108870001365536593654FF400226A61AA603D4A0F
:108880004FF4907151621363936402F53422803285
:108890004FF4905191604FF48021516001F5905157
:1088A0005161354A40F20311116051609160D1600D
:1088B000116151619161D161304900224A613049B1
:1088C0000B614B618B618B6601F5322101F5807183
:1088D0008E604E6103600826C360134611460A206D
:1088E0002A46B4461F46A646C4F804C00197019D17
:1088F000B5F57A7F2AD3DEF81050A660ED0748BFA1
:1089000001310197019DB5F57A7F23D3DEF8105030
:10891000ED0758BF01330138E6D10A2919491DD1A5
:108920000A2B1BD101230B700D4B4FF4E061196032
:10893000D96003F580534FF48071196001235360AF
:10894000536943F00103536103B0F0BD019D01354C
:108950000195CCE7019D01350195D3E70023E2E7BE
:108960000090044000F00F4040F00F407000000401
:1089700000A0044000B0044000C00440C0F00F401C
:1089800000D004406093FF1FF7B5104B1B78D3B1A4
:108990000F4B104D02210F46042000241E469F60FD
:1089A00058600194019AAA4209D97160B06001949B
:1089B000019AAA42F3D8019A01320192F8E7019A8A
:1089C00001320192EEE703B0F0BD00BF6093FF1FDC
:1089D00000F00F401FA10700032806D8DFE800F0D1
:1089E0000206080A1022054B5A6070472022FAE757
:1089F0004022F8E74FF08062F5E700BF00F10F403A
:108A0000032806D8DFE800F00206080A1022054B0A
:108A10009A6070472022FAE74022F8E74FF0806220
:108A2000F5E700BF00F10F4010B50021044644FAFD
:108A300001F3DB07C8B205D5FFF7CEFF01310829E6
:108A4000F5D110BDFFF7DCFFF8E708B5032813D810
:108A5000DFE800F0020C0E10002004F00FF843F2E3
:108A60007C03984294BF0020012008BD0120F4E758
:108A70000220F2E70320F0E7002008BD032817D802
:108A8000DFE800F002070C110A4B1868C0F3001071
:108A90007047084B1868C0F340107047054B1868C2
:108AA000C0F380107047034B1868C0F380607047B4
:108AB0000020704700F10F4070B5002425460126C4
:108AC000E0B2FFF7C2FF18B106FA04F31D43EDB29E
:108AD0000134082CF4D1284670BD024B1869C043FC
:108AE000C0B27047C0F00F4037B50446FFF7C4FD71
:108AF0000546FFF7C1FD401B0028B8BF40420128D2
:108B0000F7DD0020012C8DF804008DF8050010D051
:108B100007D3022C11D0030648BF60F0FF0003B05A
:108B200030BD022201A9902004F0D6F99DF804007E
:108B3000F1E7022201A99220F6E7224601A994203A
:108B4000F2E708B5082003F099FF5E280ED9104B14
:108B50001A780AB901221A70082003F08FFFA92899
:108B60000CD90C4B4FF400725A6008BD082003F07A
:108B700085FF5428F0D80022054BECE7082003F0CD
:108B80007DFF95289EBF034B4FF400729A6008BD8D
:108B90007486FF1F80F00F40034B187801380128BE
:108BA0008CBF0020012070477486FF1F034B18788C
:108BB000012806BF02221A70002070477486FF1F2A
:108BC000C0B204F0F9BEC0B204F0E4BE08B506F0CD
:108BD000EBFE05F0A9F905F059F9BDE8084006F0EB
:108BE00065BF38B5054605F0A7F808280AD900245E
:108BF0002819013405F020F9092CF9D105F050F9B4
:108C0000012038BD002038BD092105F0B5B800208D
:108C100005F042BB2249234841F23C028B5843F401
:108C200040538B50204B012119601A6802431A608F
:108C30001E4ADA601A61DA6A42F08052DA621A6811
:108C400022F001021A601A6822F000621A60184AC3
:108C50004FF40073136053609360D36013615361EA
:108C60009361D361A2F5F032116011680143116084
:108C70001049D16001F520011161D16A41F08051A4
:108C8000D162116821F001011160116821F00061C9
:108C9000116002F5E8329362D36213645364704743
:108CA00000700440000C1F8000C002400300013E21
:108CB00000B004400400513EFF2810B54FEA0043C5
:108CC00023D82B4C03F47C138AB141F000610B4391
:108CD0006363E36A002BFCDA254BDA6AD000FCD52B
:108CE000986BDA6A42F01042C0B2DA6210BD41F00D
:108CF00000410B436363E36A002BFCDAA06BE36A79
:108D000043F01043C0B2E36210BDB0F5007F17D24C
:108D1000184C03F47C135AB141F000610B436363B8
:108D2000E36A002BFCDA134BDA6AD100FCD5D7E7F3
:108D300041F000410B436363E36A002BFCDADDE79B
:108D40000D4C03F47C135AB141F000610B43636393
:108D5000E36A002BFCDA084BDA6AD200FCD5BFE7E5
:108D600041F000410B436363E36A002BFCDAC5E783
:108D700000C0024000D0024000C00A4010B5FFF71A
:108D80007BFC0446FFF778FC001B0028B8BF40427C
:108D90000628F7DD10BD07B5030A8DF805008DF82C
:108DA0000610032201A9A0208DF8043004F06EF80B
:108DB000FFF7E4FF03B05DF804FBF0B515460022B1
:108DC0008BB00F461446AC4201D10BB0F0BD0AABDC
:108DD0001344395D03F8221C531CC618F10602D057
:108DE000691E8C420DD1030A8DF80500033201A9DA
:108DF000A0208DF8043004F049F8FFF7BFFF30469B
:108E0000002301341A46DEE71FB5030A8DF80C3043
:108E1000022203AB8DF80D0000921946A02004F049
:108E200081F89DF80C0005B05DF804FB1FB5030A3E
:108E30008DF80C308DF80D0000920B46022203A92C
:108E4000A02004F06FF805B05DF804FBC0EBC00093
:108E5000072200F5B040FFF7B0BFC0EBC00007220B
:108E600000F5B040FFF7E2BF30B500238BB001AD95
:108E70001A465A550133222BFBD14FF4B044230A32
:108E80008DF8054022222946A02020348DF8043098
:108E900003F0FCFFFFF772FFB4F5803FEFD10BB09A
:108EA00030BD13B50C46C0EBC0000722694600F583
:108EB000B040FFF7BBFF9DF8002023789A4212D103
:108EC0009DF8012063789A420DD19DF80220A37885
:108ED0009A4208D1DDF80300D4F80330C31A58428F
:108EE000584102B010BD0020FBE7704773B545F252
:108EF000FF70FFF789FF552803D12C4B1B78002BFF
:108F00003DD0002145F2FF70FFF745FFFFF7ACFFB2
:108F1000402227490020FFF750FF402210462549F4
:108F2000FFF74BFF402223498020FFF746FF02ADA9
:108F300040222049C020FFF740FF002345F8043DB0
:108F40004FF4D36440F678062046042229460434C0
:108F5000FFF733FFB442F7D1002301934FF4FF64CE
:108F600040F6D8062046042229460434FFF725FFA0
:108F7000B442F7D1552145F2FF70FFF70CFF4022B4
:108F80000B490020FFF752FF402210460A49FFF725
:108F90004DFF402209498020FFF748FF4022084941
:108FA000C020FFF743FF02B070BD00BF6093FF1FFA
:108FB0000C80FF1F980901007893FF1FB893FF1FD3
:108FC000F893FF1F00000000044B9B78022B044B1A
:108FD0008CBF042203221A70704700BFD894FF1F71
:108FE000F495FF1F73B5CE4EB4787278022C3546D7
:108FF00003D90422CB4B1A70C3E1A32A00F02B83C0
:1090000000F2BB80132A00F0068258D8072A00F02D
:10901000BA812BD8022A00F0698107D8002A00F013
:109020005881012A00F05E810322E3E7052A00F05F
:10903000858100F29581042AF6D1D6F80300BA4E54
:10904000002856F82430B8BF4042984706EB840405
:109050002021E060A87804F0D9F8002840F0918140
:10906000A87806EB80062721F26836E10F2A00F087
:10907000B78115D80D2A00F0958100F2A2810C2A43
:10908000D2D13421204604F0C1F8D6F8033002468C
:10909000B078002B40F0838142F0020234211CE1C1
:1090A000112AA14B00F0AE8140F2A48103EB8403AE
:1090B000D6F803009B6998472A2102460CE11B2A37
:1090C00000F0E98130D8172A00F0BB8119D8152AA1
:1090D00000F0B38140F2A881D6F80300002888DBB5
:1090E000924B03EB8414237E012B01D004F0E8FCA7
:1090F0000028D2BF8E4A8F4A92FBF0F21521A87841
:10910000EBE0192A00F0B58140F2A4813421204619
:1091100004F07CF8D6F803300246B078002B00F05B
:10912000B78142F40062B9E7212A00F0DD8110D84E
:109130001F2A00F0B98100F2C6811C2A7FF474AFA7
:10914000D6F803102046C9B202B0BDE8704004F062
:109150004DB98C2A00F0D781A22A00F073827F2AB1
:109160007FF462AFD6F80330022B3FF642AF6E4B6E
:109170001C44F37884F8243003E1B82A00F0EA8232
:1091800050D8AB2A00F0AD8225D8A72A00F08E82F5
:1091900013D8A52A00F0718240F26682204604F0BE
:1091A000F0F9D6F80310C9B2002840F07982B078FF
:1091B00002B0BDE8704004F0ADB8A92A00F0888282
:1091C00040F27D82D6F803102046C9B202B0BDE855
:1091D000704004F02BBAB12A00F09E8210D8AD2A5C
:1091E00000F09182C0F08682AE2A7FF41DAFD6F8DF
:1091F00003102046C9B202B0BDE8704004F039BA8D
:10920000B52A00F08E81B62A00F08F82B32A7FF44F
:109210000BAFD6F803102046C9B202B0BDE87040CB
:1092200004F05AB9C92A00F09F812DD8BC2A00F059
:10923000BB8219D8BA2A00F09F8240F29482D6F8F5
:1092400003102046C9B204F0C5FA0021B07803F03B
:10925000DDFFD6F803100246B078002900F0A182A5
:1092600042F00402002138E0C22A00F06881C32ADB
:1092700000F06F81C12A7FF4D7AE2C4B03EB84142E
:10928000D6F8033023727CE0D22A00F0838110D814
:10929000CC2A00F09282D12A00F07481CA2A7FF48D
:1092A000C3AE224BD6F8032003EB84135A83204627
:1092B00032E1D62A00F07581FF2A00F08681D42A97
:1092C0007FF4B2AE194B03EB8414D6F8033023625B
:1092D00057E0D6F803202D21204602B0BDE87040AB
:1092E00003F050BFD6F803202121F5E7D6F803306C
:1092F000002BC8BF01222021204603F043FFB47891
:109300000D4BD6F8030001221A55074B002853F8DD
:109310002430B8BF4042984727210246DCE700BF0F
:10932000D894FF1FF495FF1F7886FF1F7893FF1FC7
:10933000B50010000024F4004E93FF1FB84BD6F880
:10934000030000221A55B74B03EB84039B6998472F
:10935000B54B43F82400B078262153F82020BCE711
:109360001021204603F052FF0346DAB2B078019292
:10937000F278D2080092C3F307430022102103F0D1
:10938000AFFE02B070BD1021204603F03FFFF2781F
:109390000346D208B0780192C3F30722EAE722F02D
:1093A00002027BE63421204603F030FFD6F803307A
:1093B0000246B07813B942F001026FE622F00102D2
:1093C0006CE63421204603F021FFD6F80330024634
:1093D000B07813B142F0100260E622F010025DE6B0
:1093E000904BD6F8030003EB84039B699847242134
:1093F000024671E753F82430D6F803009847252138
:10940000024669E703EB8403D6F803009B6998479B
:109410002821024660E7834BD6F8030053F8243036
:1094200098472321024657E77E4BD6F8030053F8AE
:10943000243098472B2102464EE7D6F803202C21F2
:109440004AE7784BD6F8030053F824309847332185
:10945000024641E73421204603F0D8FED6F8033017
:109460000246B07813B142F0080217E622F0080273
:1094700014E63421204603F0C9FED6F80330024634
:10948000B07813B142F0040208E622F0040205E6C7
:1094900022F4006202E6D6F803102046C9B202B0F8
:1094A000BDE8704003F090BF1021204603F0AEFEEF
:1094B000F3780246D1B2C2F30722B078019100924C
:1094C00003F00F0359E76E21204603F09FFEF37867
:1094D000B4780193337903F0030300930022C0F3BF
:1094E00007436E2120464AE76E21204603F08EFE98
:1094F0000246D1B2C2F30722F378B078019100920C
:109500006E2100223BE7D6F80310C1F10801204686
:10951000C9B203F035FFB07802B0BDE8704003F087
:109520003BBDD6F803000028FFF663AD3D4B53F872
:10953000243098473D4B03EB8414206121E7394BDD
:10954000D6F8030053F824309847A401374B18513C
:1095500017E7344BD6F8030053F824309847334BC1
:1095600003EB841460600CE73821204603F04EFEC4
:10957000D6F8033000F4806223F480631A43382164
:10958000B078AAE6D6F80310204602B0BDE87040D5
:1095900003F0A1BD254BD6F8032003EB8413DA6159
:1095A00085E6D6F8030006F0E7FB1BA3D3E900230A
:1095B00006F072FD41EC100B07F046F951EC100B70
:1095C00006F0DAFE1121024686E6D6F803309BB19A
:1095D000012B7FF40EAD154A02EB84121376114B6A
:1095E000134A43F8242003EB8404124BA362124B6A
:1095F000A361124B6363C4E60C4A02EB8412137638
:10960000084B0F4A43F8242003EB8404A262A261B2
:109610006263B6E6AFF300802D431CEBE236FA3FFF
:10962000D494FF1F7886FF1FC894FF1F7893FF1FF5
:1096300049DA0000C1DA000091DA000009DB00001D
:1096400041DB0000D6F803102046C9B202B0BDE8E5
:10965000704003F071BED6F803102046C9B202B0C4
:10966000BDE8704003F0D4BED6F803102046C9B25E
:1096700002B0BDE8704003F0EFBE204603F081FF6A
:10968000D6F80310C9B228B9B07802B0BDE870406E
:1096900003F020BFB07802B0BDE8704003F0EEBE2A
:1096A000B07802B0BDE8704003F002BFD6F80310F6
:1096B0002046C9B202B0BDE8704003F011BED6F832
:1096C00003102046C9B202B0BDE8704003F0E1BF0C
:1096D000D6F803102046C9B202B0BDE8704003F0CE
:1096E00093BFD6F803102046C9B202B0BDE870405F
:1096F00003F078BFD6F803102046C9B202B0BDE827
:10970000704003F0A5BFD6F803102046C9B202B0DE
:10971000BDE8704003F0CFBFD6F803102046C9B2B1
:1097200002B0BDE8704003F03DBED6F8030000284B
:10973000FFF65FAC254B03EB8414237E012B01D095
:1097400004F0BEF90028CABF214A224A92FBF0F277
:109750001421D4E4D6F803102046C9B202B0BDE803
:10976000704003F067BED6F803102046C9B202B0BD
:10977000BDE8704003F0F2BDD6F803000028FFF604
:1097800038AC124B03EB8414237E012B01D004F080
:1097900097F90028CABF0E4A0E4A92FBF0F2132135
:1097A000ADE422F0040298E5D6F803102046C9B2D1
:1097B00002B0BDE8704004F01DB8D6F80310204692
:1097C000C9B202B0BDE8704003F0BCBF7893FF1F80
:1097D0000024F400B500100038B5BE4A9078022885
:1097E000144600F0EE80032800F0F280002840F0DC
:1097F000DC8153784D2B00F0A1803AD8452B79D0ED
:1098000016D8412B6DD004D8402B63D00322B24B25
:109810005EE0422B69D0442BF8D1B049D2F8033036
:1098200041F81C3F04221C20BDE83840FFF7C5BAB0
:10983000492B6CD014D8462B61D0472BE6D1A74DCD
:10984000D2F803302946042241F8083F0820FFF7E8
:10985000B4FA2A8A29896879BDE8384003F03EB90C
:109860004B2B60D04C2BD1D19C4BD17899700220DE
:1098700033E0542B00F0838018D8512B6AD008D8DD
:109880004F2B60D0502BC1D1944BD17899751620B5
:1098900023E0522B6BD0532BB8D1904DD2F803302C
:1098A0002946042241F8103F1020D0E7842B7ED0B7
:1098B00008D8552B6FD0832BA8D1894BD2F8032021
:1098C0001A6438BD852B77D0FF2B9FD1D278854B7A
:1098D0001A7038BDD17845F2FF70BDE83840FFF707
:1098E0005ABA7E4BD1781970F7E77C4BD178597012
:1098F0000120F2E7794BD17859710520EDE77749DE
:10990000D2F8033041F80C3F04220C208CE7D278C7
:10991000724B1AB9DA75D97D1720DEE76E4901223C
:10992000DA754A60F7E76D4CD178E1700320FFF7F4
:1099300032FAE078BDE83840FEF714BF674BD178C3
:1099400059751520C9E7D2F80310644BC9B259768E
:109950001920C2E7614D2A7DD20704D5E378DB07E1
:1099600001D4FFF781FAE17829751420B5E75B4946
:10997000D2F8033041F8203F0422202054E7D2F8E7
:109980000330012B00F211815449D37801F81A3FBA
:1099900001221A2048E7D2F80330012B00F205819A
:1099A0004E49D37801F81B3F01221B203CE74E4B68
:1099B000D2F803201A6038BD494BD2F803205A640C
:1099C00038BD5178494BD2F8032043F8212038BDE7
:1099D00053782E2B3FF61AAF01A252F823F000BFA6
:1099E0009D9A0000AF9A0000C19A00000D980000F7
:1099F0000D9800000D9800000D9800000D980000D3
:109A00000D980000F59A0000FF9A0000099B0000E5
:109A10000D9800000D9800000D9800000D980000B2
:109A20000D9800000D9800000D9800000D980000A2
:109A30000D9800000D9800000D9800000D98000092
:109A40000D9800000D9800000D980000139B000079
:109A50001F9B00002B9B0000379B0000439B0000D6
:109A60004F9B00000D9800000D9800000D9800001D
:109A70000D9800000D9800000D9800005B9B000001
:109A8000659B00006F9B0000799B0000839B00009A
:109A90008D9B0000979B0000A19B0000144BD4F805
:109AA00003201A60FEF7E8FD0D4B986438BD104B9B
:109AB000D4F803205A60FEF7DFFD094BD86438BDA7
:109AC0000B4BD4F803209A60FEF7D6FD044B1865C3
:109AD00038BD00BFD894FF1FF495FF1F0C80FF1FF7
:109AE0007886FF1FEE95FF1FF095FF1F0096FF1F62
:109AF0004894FF1F2E4BD4F80320DA6038BD2C4B5E
:109B0000D4F803201A6138BD294BD4F803205A61D8
:109B100038BDD4F80330264ADBB2137638BDD4F80A
:109B20000330234ADBB2D37638BDD4F80330204A61
:109B3000DBB2537638BDD4F803301D4ADBB213775D
:109B400038BDD4F803301A4ADBB2937638BDD4F866
:109B50000330174ADBB2537738BD154BD4F80320D6
:109B60001A6238BD124BD4F803205A6238BD104B2C
:109B7000D4F803209A6238BD0D4BD4F80320DA6282
:109B800038BD0B4BD4F803201A6338BD084BD4F80A
:109B900003205A6338BD064BD4F803209A6338BDBE
:109BA000034BD4F80320DA6338BD04222FE600BF4C
:109BB0004894FF1F2DE9F043C64EC74F32787A70A4
:109BC00064233B70212AD6F803307B6085B035468C
:109BD0003C4601F0C58200F2E8800E2A00F07C8746
:109BE0005ED8072A00F0EF8539D8032A00F02C82CE
:109BF00008D8012A00F0B581022A00F0EE81022384
:109C00002370E4E1052A00F0468340F23A82B078FE
:109C10007378022800F2DE81A42B00F08A8500F21E
:109C2000CA83122B00F0E28400F26683082B00F056
:109C3000AD8400F24183032B00F0868400F22E8372
:109C4000012B00F07F8440F26884A44B03EB800377
:109C500027219D6A03F0DAFAA84700F061BC0A2ABE
:109C600000F0D28507D8082A00F0B085092AC6D1AD
:109C7000FFF7B2FDABE10C2A00F0E58640F2CB869F
:109C8000B078022800F2A6817378012B00F0F386E9
:109C9000C0F0ED86022B00F0F28603233B7096E1C4
:109CA000182A01F075802BD8142A00F0BE8715D829
:109CB0000F2A00F03087132AA1D17178884A092928
:109CC00000F28787DFE811F082078E07910794077B
:109CD00098079F07A207A507A8079D07162A01F066
:109CE000488040F2C3877D4AD16D072900F26F8119
:109CF000481C02EB8101D065906D0866936566E1B2
:109D00001C2A01F03F8122D81A2A01F05F8041F21B
:109D10004C80724C94F8812072B95E1C04BF704B69
:109D20001B680A205843C4F88400FEF7A5FC0123F1
:109D3000C4F8880084F881306B78042B00F24781E6
:109D4000DFE813F055089608C408F2086B081F2ACC
:109D500001F04D8101F2AA811E2A7FF450AF727882
:109D6000142A00F26886B078022801F2118102EB11
:109D700042045C4D044445F824305B4B9B7E002B31
:109D800000F02581002A00F02281032111FB02014D
:109D90000C23013A5A4302F5D363042205EB8101F7
:109DA00002FB0030FFF709F811E1802A01F0B482CC
:109DB00044D8402A01F0988229D8242A01F02E8222
:109DC0000CD8222A01F02282232A7FF418AF444BB8
:109DD0001B68C6F80330FFF7FFFCF8E0262A01F005
:109DE0005B82C1F04E82272A7FF409AFB278022A43
:109DF00000F2F0807378142B00F21D8603EB43030E
:109E00001344374A1168374A42F82310DFE0442AE6
:109E100001F0768207D8422A01F06E8241F2688210
:109E200002F033F9D3E0462A01F07282C1F06C826D
:109E3000472A7FF4E4AE02F02CF9C8E0872A01F04B
:109E4000128357D8832A01F093820AD8812A01F01D
:109E50006982822A7FF4D3AE204B022283F85420F9
:109E6000B5E0852A01F0B7821F4A41F2A1821F495D
:109E70001F4C01250D70B3F5C05F9178217081F002
:109E8000B082127D12EA050641F0AB82184602A9A3
:109E9000FEF7E3FF9DF8083063709DF80930A3706A
:109EA0009DF80A30E3709DF80E3023719DF80D3057
:109EB00063719DF80C30A3719DF80B30E37126722D
:109EC0002B46E15C227A01330A44082B2272F8D136
:109ED0007DE000BFD894FF1FF495FF1F7886FF1F19
:109EE000E095FF1FE494FF1F0C80FF1FE495FF1F08
:109EF000E595FF1F8C2A01F0FE821FD8892A01F008
:109F0000DF82C1F078828A2A7FF479AE72789D4B25
:109F1000002A41F0ED821A709B4AEB7813709B4A3D
:109F200092F870119A4A11709A4900220A709A495F
:109F30000A709A4A11780B43137048E0F22A01F034
:109F40004983FF2A01F08B838D2A7FF458AE727803
:109F5000032A01F23B83DFE812F00E0BF50A270B10
:109F6000350BB078022835D88D4B8E4E00241C540A
:109F70008D4B1C54335C3BB18C4B262153F8202075
:109F800003F000F9AB78F454AC78894BD5F80300B2
:109F900001261E557D4B002853F82430B8BF40429F
:109FA000984727210246204603F0ECF8D5F8033005
:109FB000A878002BD8BF02224FF00003D6BF019231
:109FC0008DE8480000931A46202103F089F805B077
:109FD000BDE8F08304232370F9E7B0780228F9D8AC
:109FE0006F4B704E00241C546F4B1C54335C3BB1C0
:109FF0006E4B262153F8202003F0C4F8AB78F454BC
:10A00000AC786B4BD5F8030001261E555F4B00283A
:10A0100053F82430B8BF40429847272102462046D3
:10A0200003F0B0F8D5F80330A878002BC8BF02229F
:10A030004FF00003C6BF019200938DE848001A4616
:10A04000202103F04DF8C2E7B0780228C2D802F010
:10A0500083FCB078564B01221A542721002203F0CA
:10A0600091F800240223B0780193224623460094FD
:10A07000202103F035F8B378494AD4544A4AD454DD
:10A08000A5E7B078022802D97278022A9FD1444A03
:10A090004FF0000802F80080434A02F800806A7816
:10A0A000012A2FD005D3022A00F0848003232370D5
:10A0B0008DE73F4C235C4BB1344B03EB80032721EE
:10A0C000DA6803F05FF8AB7804F80380A878354CC1
:10A0D000235C43B1354B262153F8202003F052F87E
:10A0E000AB780022E254D5F80320A8782D2103F0A4
:10A0F00049F80023A878019300931A46202102F022
:10A10000EFFF64E7214F3A1892F82420012A33D058
:10A110002DD3022A32D0A878254E335C43B107EB09
:10A1200080032721DA6803F02DF8AB780022F2547F
:10A13000A8781C4E335C43B11C4B262153F82020D9
:10A1400003F020F8AB780022F254D5F80360A87829
:10A15000464432462D2103F015F80023A8780193D8
:10A1600000931A46202102F0BBFF66602FE72D21E5
:10A1700003F04CF88046CEE72121F9E702F0A8FF72
:10A18000F8E700BF4093FF1F5293FF1F7886FF1F21
:10A190009894FF1F5193FF1FD794FF1F4193FF1FF8
:10A1A0004B93FF1FD494FF1F7093FF1FC894FF1F92
:10A1B0004E93FF1F142B3FF70DAF020639D54446CF
:10A1C000C84FDFF83083DFF83093AB782341DB07EB
:10A1D0002BD5E35DE6B243B1C34B272153F82420CE
:10A1E000304602F0CFFF0023E35514F808304BB19E
:10A1F000BE4B262153F82420304602F0C3FF002333
:10A2000004F80830D5F8033003EB430323442D2131
:10A2100059F82320304602F0B5FF00230193009344
:10A220001A462021304602F05BFF0134032CCCD1CA
:10A23000CDE602283FF6CEAEAA4C235C4BB1AC4B28
:10A2400003EB80032721DA6802F09CFFAB7804F867
:10A250000380A878A74C235C43B1A44B262153F874
:10A26000202002F08FFFAB780022E254D5F80330B3
:10A27000A878A14A03EB430303442D2152F823207D
:10A2800002F080FF0023A878019300931A46202152
:10A2900002F026FF9BE6FEF7A5FE98E6052B00F0F0
:10A2A0006181C0F05881062B00F06481072B00F01B
:10A2B00068810323237034E10D2B00F081810BD8DA
:10A2C0000A2B00F06C81C0F067810B2B00F07181CC
:10A2D0000C2BEED1342163E10F2B00F07981C0F01B
:10A2E0007181102B00F07B81112BE2D1804B03EBAD
:10A2F000800328215D6BADE41C2B00F0A78133D8CF
:10A30000172B00F08A8122D8142B00F07D81C0F039
:10A310007481152B00F07F81162BCAD1152102F014
:10A3200075FF0028D5BF6FF07F43744B636093FBCC
:10A33000F0F0AA78724BC8BF606003EB82131B7EFB
:10A34000002B40F0EE80606803F07EFBE8E0192B04
:10A3500000F07081C0F068811A2B00F071811B2B16
:10A36000A7D103F000F9DBE0212B00F080810FD8AA
:10A370001E2B00F07681C0F06C811F2B00F07181E4
:10A38000202B96D16E2102F041FFC0F30900C7E0F7
:10A390008C2B00F0718106D87F2B8AD1544B184446
:10A3A00090F8243003E1A22B00F0C081A32B80D1D0
:10A3B00003F0E7F8B4E0BB2B00F0EF8148D8AD2BF9
:10A3C00000F0DC8119D8A82B00F0CC8107D8A62B8F
:10A3D00000F0BD8140F2B08103F090F8A0E0AA2B1C
:10A3E00000F0C681C0F0C181AB2B00F0C481AC2B62
:10A3F0007FF45FAF03F086F992E0B52B00F0418166
:10A4000015D8B12B00F0BD8105D8AE2B7FF451AF2C
:10A4100003F07FF984E0B32B00F0B681B42B7FF416
:10A4200048AF6F2102F0F2FEC0F3044078E0B82B91
:10A4300000F0AD8104D8B62B7FF43BAF14216EE75A
:10A44000B92B00F0A781BA2B7FF433AF132166E755
:10A45000CA2B00F0378120D8C22B00F01C810FD806
:10A46000BD2B00F0A081C0F09B81BE2B00F09D8130
:10A47000C12B7FF41EAF224B03EB8010037A96E0D2
:10A48000C42B00F01981C0F00E81C52B00F018819B
:10A49000C92B7FF40EAF382140E0D12B00F02B8187
:10A4A00014D8CE2B00F0138105D8CC2B7FF401AF4C
:10A4B00003F0B0F934E0CF2B00F00B81D02B7FF408
:10A4C000F8AE6F2102F0A2FE000E29E0D42B00F0BE
:10A4D000158117D8D22B7FF4ECAE094B03EB80101B
:10A4E000C36964E04E93FF1F8486FF1FC894FF1F5B
:10A4F0007886FF1FD494FF1FE494FF1F0024F4000C
:10A500007893FF1FD62B00F0FE80FF2B7FF4D1AE97
:10A51000B34B03EB8010037E49E02D2102F076FE61
:10A520006060B04B1B78002B3FF451ADAE4B6268BE
:10A530001A60AE4B002A40F041811A6842F00802CE
:10A540001A6044E52121E9E7A94B03EB80032221AE
:10A550009D6AFFF77FBBA64B03EB8000836AC06850
:10A560009847DDE7A24BA34A03EB800352F8200093
:10A570005B6BF5E7102102F049FEC0F30720C00035
:10A58000CEE7102102F042FEC0B2F8E7352102F01A
:10A590003DFEC0F34020C3E703F03EFAC0E735219B
:10A5A00002F034FE10F0020F0CBF012300236360A1
:10A5B000B7E7352102F02AFEC04300F00100AFE703
:10A5C0003421F7E7342102F021FEC0F30010A7E7A1
:10A5D000874B03EB800324215D6BFFF73BBB844B70
:10A5E00003EB800325219D6AFFF734BB804B03EB0F
:10A5F00080032A215D6BFFF72DBB7D4B03EB8003AE
:10A6000023219D6AFFF726BB794B03EB80032B21A7
:10A610009D6AFFF71FBB2C2180E7754B03EB80037E
:10A6200033219D6AFFF716BB342102F0EFFDC0F322
:10A63000C00075E7342102F0E9FDC0F380006FE748
:10A64000342102F0E3FDC0F3C02069E702F092FF7D
:10A6500066E7674B03EB80039D6A01F029FDFFF776
:10A66000FBBA102102F0D2FDC0F3034058E76E217F
:10A6700002F0CCFD001453E702F067FFC0F10800C0
:10A680004EE75B4A564B03EB801302EB8000826A75
:10A690001869904744E7564B5149820103EB80000B
:10A6A000836A88585CE7524A4D4B03EB801302EBF8
:10A6B0008000826A5868ECE74F4B53F8203076E709
:10A6C0004E4BFAE7464B03EB8010438B6FE76F214D
:10A6D00059E64B4B195C00227A6009B1012179607F
:10A6E0001A54484B1A5C1AB1626842F00202626066
:10A6F00000221A5415E702F0EBFC11E7384B03EB8C
:10A700008010036A53E7112102F080FD05F034FB4D
:10A7100031A3D3E9002305F095FB41EC100B05F0C4
:10A72000FFFF51EC100B05F027FEF9E602F0FFFEEB
:10A73000F6E602F034FFF3E602F023FF18B9B07832
:10A7400002F047FFECE6B07802F030FFE8E602F0F6
:10A7500018FF18B9B07802F0E3FEE1E6B07802F035
:10A7600031FFDDE602F0E0FFDAE602F0BDFFD7E6FA
:10A7700002F0C1FFD4E602F0B0FFD1E602F0DBFF49
:10A78000CEE602F0E9FECBE602F025FFC8E602F0D5
:10A79000FFFEC5E602F0D2FEC2E603F057F8BFE6C0
:10A7A00003F05BF8BCE67121B8E6002102F02EFD53
:10A7B00010F004003FF4B4AE0123F8E61A6822F06A
:10A7C00008021A6003E4FEF7FFFB00E4FEF7FCFB5F
:10A7D000FFF7FDBBAFF300802D431CEBE236FA3FE1
:10A7E0007893FF1FEF95FF1FE095FF1FE094FF1F79
:10A7F0007886FF1FC894FF1F3493FF1F3C94FF1FF0
:10A800007093FF1F4B93FF1FB378022B00F0B780AC
:10A81000032B00F0B980002B40F0F5807378502BAB
:10A8200000F0828028D8462B6FD010D8422B66D0FB
:10A8300006D8402B48D0412B5DD00323237048E03D
:10A84000442B5FD0452BF8D1984B5B7955E04B2BCF
:10A8500061D009D8472B5BD0492BEED1934BDB7DE0
:10A86000003318BF012348E04D2B5AD056D34F2B4D
:10A87000E3D18E4B5B7E40E0802B64D012D8532B0B
:10A8800058D006D8512B52D0522BD6D1874B1B6AA9
:10A8900033E0552B54D050D3562BCED1834B93F865
:10A8A00024302AE0832B59D006D8812B4FD0822B1D
:10A8B000C3D17F4B9B6D20E0852B55D051D3FF2B0F
:10A8C000BBD17C4B1B78CBE745F2FF70FEF79CFABF
:10A8D0007860794B1B78002B3FF479AB774B62683B
:10A8E0001A60774B002A40F090801A6842F0080204
:10A8F0001A60FFF76CBB6D4B1B786360E9E76B4B2D
:10A900005B78FAE7694BDB69F7E7684BDB68F4E7EC
:10A91000664B9B68F1E7654BDB78EEE7634B9B7812
:10A92000EBE7624B5B7DE8E7604B9B7DE5E75F4BC8
:10A930001B7DE2E75D4B1B69DFE75C4B9B7EDCE741
:10A940005A4BDB7ED9E75A4B93F85430D5E7584B36
:10A9500093F854301E1F73427341CEE7544B1B6C67
:10A96000CBE7584B1B68C8E7514A5748536C43F232
:10A97000390100FB0313536423F00043BDE77278F1
:10A98000524B53F82230B8E77378282B2CD013D8C9
:10A99000022B27D006D81BB3012B7FF44EAF4C4BB4
:10A9A0005B68AAE7092BFFF448AF0B2B91D9272B43
:10A9B0007FF443AF464B6AE72B2B1BD007D8292BDC
:10A9C00015D02A2B7FF439AF414BDB6A95E72D2B4D
:10A9D00016D012D32E2B7FF430AF3D4BDB6B8CE7C0
:10A9E0003B4BBFE73A4B94E7394B5B6A85E7384B03
:10A9F0009B6A82E7364B1B6B7FE7354B5B6B7CE7D3
:10AA0000334B9B6B79E7042318E71A6822F008029E
:10AA10001A60FFF7DCBAB378022B10D170783728B0
:10AA200009D800F5FF702B49800004220144FEF78D
:10AA3000C4F9FFF7CCBA03232370FFF7C8BA042385
:10AA40003B70FFF7C4BAB378022B0CD1707837286B
:10AA5000F1D800F5FF701F49800004220144FEF781
:10AA6000E5F9FFF7B4BA04233B70FFF7B0BA01F081
:10AA70006BFFFFF7ACBA01F06FFFFFF7A8BA01F068
:10AA800073FF0D4B78601B78002B3FF4A0AA0B4B93
:10AA900018600B4B1A6820B942F008021A60FFF7E1
:10AAA00096BA22F008021A60FFF791BA0C80FF1FD5
:10AAB0007886FF1FEE95FF1FEF95FF1FE095FF1FA4
:10AAC000E094FF1FF095FF1F6D4EC6410096FF1FDB
:10AAD0004894FF1F088EFF1FB278022A17D17078A2
:10AAE000072808D81BB9FDF78BFFFFF770BAFDF7F1
:10AAF00073FFFFF76CBAFF287FF469AA5D1C0ABFD9
:10AB00009E4BD8B21878FDF78FFFFFF760BA042389
:10AB10003B70FFF75CBAB378012B2AD023B1022B2C
:10AB20004AD004233B700FE07078082803D8FDF763
:10AB30008CFF606008E00A2816D1914B1B6983F4F2
:10AB40000073C3F340237B608E4B1B78002B3FF4D4
:10AB50003EAA8A4B62681A608B4B8ABB1A6842F025
:10AB600008021A60FFF733BAFF28EDD1FDF7A4FF02
:10AB7000DFE77078092802D001F080FFD9E70020D4
:10AB8000FDF7B2FF05460120FDF7AEFF06460220A5
:10AB9000FDF7AAFF8642D4BF002301239D4209DDB1
:10ABA000331C18BF01231BB986423546B8BF054682
:10ABB0006560C9E7031CF4E77078FDF75FFFB8E74D
:10ABC0001A6822F008021A60FFF701BA10681844E8
:10ABD000106012686C4B12BB1A6842F008021A60CF
:10ABE000FFF7F5B91068C01AF2E710685843EFE7AD
:10ABF000106890FBF3F0EBE7116891FBF3F003FBB7
:10AC000010131360E5E710681840E1E71068184377
:10AC1000DEE710685840DBE71368DB43F1E71A68AA
:10AC200022F008021A60FFF7D2B9544A1168564A56
:10AC30008B4213680BDA23F0030343F00403136021
:10AC4000136871B943F008031360FFF7C0B90BBF75
:10AC500023F0060323F0050343F0010343F002034E
:10AC6000EDE723F008031360FFF7B1B972780C2AFF
:10AC70003FF6ADA9DFE802F0071019222B343E475A
:10AC80005059626B7400404A126814077FF59FA9FF
:10AC90003E4A9365FFF79BB93B4A126810073FF5A0
:10ACA00096A93A4A9365FFF792B9374A1268D107D5
:10ACB0007FF58DA9354A9365FFF789B9324A126845
:10ACC000D2073FF584A9314A9365FFF780B92E4A30
:10ACD000126857077FF57BA92C4A9365FFF777B970
:10ACE000294A126812F0050F3FF471A9274A9365AB
:10ACF000FFF76DB9244A126896077FF568A9234AC1
:10AD00009365FFF764B9204A126895073FF45FA97D
:10AD10001E4A9365FFF75BB91B4A1268D4067FF59C
:10AD200056A91A4A9365FFF752B9174A1268900656
:10AD30007FF54DA9154A9365FFF749B9124A126884
:10AD400051067FF544A9114A9365FFF740B90E4AB1
:10AD5000126812067FF53BA90C4A9365FFF737B9D5
:10AD6000094A1268D7057FF532A9084A9365FFF7AB
:10AD70002EB9064A9365FFF72AB900BFE095FF1F79
:10AD800080F00F40EF95FF1FE094FF1F7886FF1FB4
:10AD9000C04AD36D002B3FF41AA9013BD36502EBE7
:10ADA00083031B6E9365FFF712B973782E2B04D8BB
:10ADB000B94A0121D154FFF70AB9FF2B7FF43BAE0A
:10ADC000B44B012283F88020FFF701B973782E2B52
:10ADD00004D8B14A0021D154FFF7F9B8FF2B7FF412
:10ADE0002AAEAC4B002283F88020FFF7F0B8FDF7C5
:10ADF00043FCD4F88830C01A0028D4F88430B8BF97
:10AE00004042984295BFA36D002303F1FF3384F8BD
:10AE1000813098BFA365FFF7DAB8A87801F0A4FDE8
:10AE200040B99E4A84F88100136823F01003136030
:10AE3000FFF7CDB8D4F88430ABB1FDF71DFCD4F8E2
:10AE40008830C01A0028D4F88430B8BF40429842F5
:10AE500009D9924A002384F88130136843F0100323
:10AE60001360FFF7B4B8A36D013BA365FFF7AFB85C
:10AE7000A878352102F0CAF910F4007509D0874A84
:10AE8000002384F88130136823F010031360FFF768
:10AE90009EB8D4F88430A3B1FDF7EEFBD4F8883027
:10AEA000C01A0028D4F88430B8BF4042984208D96C
:10AEB0007A4A84F88150136843F010031360FFF757
:10AEC00086B8A36D013BA365FFF781B8A87835214B
:10AED00002F09CF910F0010509D0704A002384F8B3
:10AEE0008130136823F010031360FFF770B8D4F8B3
:10AEF0008430A3B1FDF7C0FBD4F88830C01A002815
:10AF0000D4F88430B8BF4042984208D9634A84F8E4
:10AF10008150136843F010031360FFF758B8A36D16
:10AF2000013BA365FFF753B8A878352102F06EF90D
:10AF300010F0020509D0594A002384F881301368C3
:10AF400023F010031360FFF742B8D4F88430A3B1A4
:10AF5000FDF792FBD4F88830C01A0028D4F884306A
:10AF6000B8BF4042984208D94C4A84F881501368CF
:10AF700043F010031360FFF72AB8A36D013BA365EC
:10AF8000FFF725B8434B002283F85420FFF71FB882
:10AF9000FF287FF41FA8424E3AB300244FF0030865
:10AFA0000C27687818FB00410138784300F5D3601E
:10AFB00000EB8400042206EB81010134FDF7FDFE65
:10AFC000032CEED1FFF703B861197819042231443C
:10AFD0000435FDF7F2FE0C2DF6D10C34FC2C3EF4BA
:10AFE000F6AF002504F28C67EEE70C24F9E77378DE
:10AFF000142B3FF620ADB278022A1BD803EB430393
:10B000001344274A52F82320264B7A601B78002BE2
:10B010003EF4DDAF244B1A60204B2AB91A6842F087
:10B0200008021A60FEF7D3BF1A6822F008021A60FD
:10B03000FEF7CDBFFF2A7EF4CDAF194E3BB30024FF
:10B040004FF003080C27687818FB0041013878435B
:10B0500000F5D36000EB8400042206EB810101348B
:10B06000FDF7E4FE032CEED1FEF7B1BF61197819AC
:10B07000042231440435FDF7D9FE0C2DF6D10C34F1
:10B08000FC2C3EF4A4AF002504F28C67EEE70C2400
:10B09000F9E700BF7886FF1F9994FF1FE094FF1F18
:10B0A000E494FF1FEF95FF1FE095FF1F7678142EA5
:10B0B0003FF6C1ACAF7838062AD5A64FDFF89882A4
:10B0C0000024AB782341D90709D56E782121E0B25D
:10B0D00002F09CF806EB4606264447F8260098F84E
:10B0E0001A3083B16B7873B1032111FB03410C203B
:10B0F000013B584300F5D360042207EB810100EBCC
:10B100008400FDF75AFE0134032CDAD1FEF75FBF4D
:10B11000022F3EF65FAF2121384602F077F88E4BC2
:10B120008C4C9B7E06EB46063E4444F82600002BE2
:10B130003EF44DAF6A78002A3EF449AFA878032167
:10B1400011FB02010C23013A534303F5D36304229C
:10B1500004EB810102FB0030FDF72FFEFEF737BF45
:10B1600072787E4B0A2A0CD8DFE802F006151A1F07
:10B17000252D32373C41450079491A6809680A444F
:10B180001A601A68774B002A3AD11A6842F008020E
:10B190001A60FEF71CBF72491A680968521AEFE775
:10B1A0006F4A196812684A43EAE76D491A680968E4
:10B1B00092FBF1F2E4E76A4A1868116890FBF1F239
:10B1C00001FB1202DCE766491A6809680A40D7E702
:10B1D00063491A6809680A43D2E761491A6809682D
:10B1E0004A40CDE75E490A68D2430A60C9E7196858
:10B1F0005B4A1160C5E75A4A196810681860F8E799
:10B200001A6822F008021A60FEF7E1BE534B1B6871
:10B21000C6F80330FDF7E6FEFEF7D9BE7378052BBE
:10B220003EF6D5AEDFE803F0030A11181F264D4A9B
:10B23000136803F00F031360FEF7C9BE494A136891
:10B2400023F010031360FEF7C2BE464A136823F0D2
:10B2500020031360FEF7BBBE424A136823F040038D
:10B260001360FEF7B4BE3F4A136823F080031360F7
:10B27000FEF7ADBE3B4A136823F480731360FEF7FC
:10B28000A6BE71782E293FF6D6AB374A02EB810273
:10B29000C2F88C30FEF79BBE334B304AD3F84811CE
:10B2A00011602F4AD3F84C111160D3F850219A65E0
:10B2B0002C4AD3F854111160D3F8582183F8812017
:10B2C000D3F85C21C3F88820D3F86021C3F8842028
:10B2D00093F86411254A505C08B1012050540022B3
:10B2E00083F86821FEF773BE00F0C0FEFEF76FBE64
:10B2F00000F0BDFEFEF76BBE00F0C6FEFEF767BEB7
:10B3000000F0C4FEFEF763BE00F0C1FEFEF75FBEB4
:10B3100000F0BEFEFEF75BBE134B002283F8542004
:10B32000FEF755BE72782AB1012A09D003233B707B
:10B33000FEF74DBE0C4B012283F85420FEF747BEAA
:10B34000B3F5C05FBEF446AE074981F854208B6563
:10B35000FEF73DBEE494FF1F0C80FF1FE095FF1F2A
:10B36000FC95FF1FE094FF1F7886FF1F9994FF1F35
:10B37000C04AC148002382F8803082F8683102F167
:10B380008C044FF0FF35194644F82350C154013363
:10B390002F2BF9D1B94B82F854101960B84B916535
:10B3A0001960B84BD16582F881101960FEF70FBEA5
:10B3B000127D92070BD4B3F5C05FBEF40BAEAD4A5D
:10B3C000042182F85410C2F86C31FEF700BE082345
:10B3D0003B70FEF7FCBDA74B002283F85420FEF71C
:10B3E000F6BD2B460022E2540133082BFBD1237813
:10B3F0002372FEF7ECBD7378012B19D005D3022B15
:10B400001FD003233B70FEF7E2BD9F4B01221A7051
:10B410009E4B9F4A9B7813709E4B196800230139FD
:10B42000013311F8010FD054082BF9D1FEF7CFBD2D
:10B430000C22FA717B718E220723BA713B71FEF7E1
:10B44000C6BD914B944801221A70904B904A9B784C
:10B450001370002301331918082B11F8091CD1545B
:10B46000F8D1FEF7B4BD7378032B3EF6B0ADDFE83C
:10B4700003F002101D227F4B93F85420FA7193F8C9
:10B480008120D3F86C31BA711A0A7A713B71FEF7D8
:10B490009EBD784B93F85420FA7193F881209B6DF0
:10B4A000BA711A0A7A713B71FEF791BD734B1B6832
:10B4B0007B60FEF78CBD724B1B687B60FEF787BD1F
:10B4C0007278002A7EF483ADB17800297EF47FADD6
:10B4D00040F2D24293427EF47AAD45F2FF70FDF71E
:10B4E0005AFCFDF7C1FC0120FDF7A2F9FEF76FBD84
:10B4F0000122FEF710BD75782DB1012D13D0032365
:10B500003B70FEF764BD042202A945F2FB70FDF713
:10B510008DFC029BD6F803209A4206BF01237B6074
:10B520007D60FEF754BDB3782A2B07D104225B4916
:10B5300045F2FB70FDF741FCFEF749BD03233B706C
:10B54000FEF745BD4B4CD4F87401002104F5BC72E4
:10B5500081423EF43CAD52F821509D4201F101057B
:10B5600020D102EB8503043B0138814214D3C4F897
:10B570007401FEF72CBD3F4AD2F8741109299DBF12
:10B58000481CC2F8740102EB8102092394BFC2F87F
:10B5900078313B70FEF71BBD53F8042F43F8042CA1
:10B5A0000131E2E72946D3E7324A0023C2F8743179
:10B5B000194602F5BC7242F8231001330A2BFAD166
:10B5C000FEF705BD0A237B60FEF701BD03233B7038
:10B5D000FEF7FDBC7378812B7EF4FCACB378922B24
:10B5E0007EF4F8ACB379A32B7EF4F4AC7379B42B6E
:10B5F0007EF4F0AC3379C52B7EF4ECACF378D62B2B
:10B600007EF4E8ACFDF703FBFDF736F80446FDF7E2
:10B6100033F8001B0028B8BF4042B0F57A7FF6DB54
:10B62000FDF704F91E4B00221A604FF0FF32C3F8F9
:10B630007021C3F87022C3F87421C3F87422C3F8D0
:10B640007821C3F87822C3F87C21C3F87C22154BFB
:10B65000154A1A600120FDF7EBF8FEF7B8BC40F27E
:10B66000D24293427EF4B3AC024B012283F8A02174
:10B67000FEF7ADBC7886FF1F9994FF1FE095FF1F72
:10B68000FC95FF1FE094FF1FE495FF1F0C80FF1F38
:10B69000E595FF1F0880FF1F00800000DB94FF1F5F
:10B6A00010E000E00080FF1F785634122DE9F84FBB
:10B6B000424B434EDFF844B100241C60414BB4655B
:10B6C0001C60414B86F881401C6006F1280906F198
:10B6D000180A0BEB84134FEA84081B7E3B4A002BAD
:10B6E0003BD13B4B46F8243049F824304AF824300B
:10B6F000E7B242F824302721384601F087FD354B68
:10B7000043F80800344B0025E5542621384601F063
:10B710007DFD324B43F80800314B3846E554013487
:10B7200001F03AFC032CD4D12E4A2B4629469046F0
:10B7300042F823100133B3F5807FF9D12A4CA37E60
:10B740003BBBE37E4BB3637DB3B3FDF725FA98B300
:10B75000012386F85430BDE8F88F244B46F8243096
:10B76000234B49F82430234B4AF82430224BBFE7BF
:10B77000791909EB0700042251440437FDF756FB01
:10B780000C2FF5D10C35FC2DDBD0002705F28C6990
:10B79000EEE70C25DFF868A0F7E74FF4FF6540F609
:10B7A000D807A5F5FF612846042241440435FDF77A
:10B7B0003DFBBD42F5D1C6E70023CAE7E095FF1F78
:10B7C0007886FF1FFC95FF1FE094FF1FAC86FF1FCC
:10B7D00041DB00008486FF1F4E93FF1FC894FF1FAC
:10B7E000D494FF1F0096FF1F0C80FF1F49DA000052
:10B7F000C1DA000091DA000009DB00007893FF1F36
:10B80000E494FF1FF7B50F4C07460E4694E803007B
:10B810008DE803000C49C1F803300C4B8A700022FC
:10B820000F704E701A70FEF7C5F9094A217882F838
:10B83000A1119DE80300636884E80300184603B083
:10B84000F0BD00BFF495FF1FD894FF1FEF95FF1FB9
:10B850007886FF1FF7B504461F4A63781370A378F4
:10B860005370E37893702379937163795371A3795B
:10B870001A4D1371E379D3700E4695E80300184B07
:10B8800000221A708DE80300FEF794F9154B1A7820
:10B890006F462B469AB9327072702A78B2706A7805
:10B8A000F270EA793271AA7972716A79B2712A7981
:10B8B000F27197E8030083E8030003B0F0BD012AAA
:10B8C000F7D10948721EF11D10F8014F02F8014F1F
:10B8D0008A42F9D1EDE700BFD894FF1FF495FF1F0E
:10B8E000EF95FF1FE495FF1FE595FF1F014B93F8B0
:10B8F000A10170477886FF1F2DE9F043994B9A4CC0
:10B900001B788FB06BB1994B1B78063BDBB2192BC0
:10B9100004D8974A22FA03F3D90702D4002384F803
:10B92000703194F87031934E5A1E012A51D89249C1
:10B93000012BCA68079214BF082307238DF818301B
:10B94000327894F8A2318DF8193000238DF81A302E
:10B95000002A33D18B688DF82030884B8DF8272052
:10B9600019788DF8211059788DF82210D9798DF831
:10B97000231099798DF8241059791B798DF82510A9
:10B980008DF8263006A801F097F9002800F01F83F3
:10B990007B4B1A789846002A00F01E81794B7A4F2B
:10B9A0001B78013B062B00F21381DFE813F0F10056
:10B9B000F10058011101110111017F01012AE1D1AA
:10B9C0007248013306AA1A44195CD171082BF8D1C8
:10B9D000D8E7032B3DD1337883BBDFF89C81674FD9
:10B9E00098F8020098F801503B7805441D447B7894
:10B9F0001D44FB791D44BB791D447B791D443B7973
:10BA00001D44FCF773FE98F80100FCF76FFE3878D0
:10BA1000FCF76CFE7878FCF769FEF879FCF766FEB7
:10BA2000B879FCF763FE7879FCF760FE3879EDB2FF
:10BA3000FCF75CFE2846FCF759FEA9E7012BA7D1CD
:10BA4000524F0025785D0135FCF750FE092DF9D1E4
:10BA50009EE7042B2BD1484FDFF82081B8787D7802
:10BA6000002301220544154488F8013088F800209D
:10BA7000C8F80430FCF73AFE7878FCF737FE98F8FF
:10BA80000000FCF733FE98F80100FCF72FFE98F851
:10BA90000700FCF72BFE98F80600FCF727FE98F845
:10BAA0000500FCF723FEEDB298F80400C0E7072B71
:10BAB00037D1337853BB304B9F7893F801802F4BAD
:10BAC0008DF800701D785878D9798DF80250474468
:10BAD0003D449A798DF80300284493F805C08DF809
:10BAE0000410014493F804E08DF805200A440CEB9F
:10BAF000020373448DF801808DF806C08DF807E0CD
:10BB00008DF808306846FDF77FF841E7012BF9D141
:10BB10001E4900235A5C0DF803200133092BF9D18B
:10BB2000F0E7082B7FF434AF144A134900230120B7
:10BB30005370107053608A7849788DF800200A4459
:10BB400002448DF801108DF802008DF803308DF855
:10BB500004308DF805308DF806308DF807308DF8FB
:10BB60000820CFE7EE95FF1F7886FF1FD894FF1FB0
:10BB700011020002E495FF1F0C80FF1FF495FF1FC8
:10BB8000D794FF1F9894FF1F5193FF1FE595FF1F48
:10BB9000AE4A397893688DF8303080238DF8313093
:10BBA0008A238DF8323000238DF833308DF834300D
:10BBB0008DF835308DF836108DF8293007218DF845
:10BBC0002A300AA8D3688DF828100B9301F074F876
:10BBD00000233B7088F80030002384F87031337004
:10BBE00094F8A03113B10120FCF722FE06A800F062
:10BBF000EFFF0646002800F04181954B9DF820207C
:10BC00001A709DF821205A709DF822209A709DF894
:10BC100023209A719DF824205A719DF825201A71CD
:10BC20009DF82620DA709DF8193084F8A231FCF7CF
:10BC300023FD884B1860884B00221A709DF818303D
:10BC4000072B0CBF0123022384F8703194F8543081
:10BC50005A1E012A4AD9052B48D0012247E0DFF8B5
:10BC6000EC913B7899F8020099F8015005440A35A7
:10BC70001D44FCF73BFD99F80100FCF737FD8020DF
:10BC8000FCF734FD8A20FCF731FD0020FCF72EFD87
:10BC90000020FCF72BFD0020FCF728FDEDB23878E2
:10BCA000FCF724FD2846FCF721FD91E7674A507810
:10BCB00093788DF80C303A788DF80D00802103448C
:10BCC0008DF80E100A338A218DF80F1013440021CD
:10BCD00003A88DF810108DF811108DF812108DF842
:10BCE00013208DF81430FCF78FFF71E700225B4BB7
:10BCF0001A7094F85430042B04D1554B19780A0665
:10BD000040F1688194F87021082A04D840F2511358
:10BD1000D340DF0701D4FDF74DFF94F87031092BB4
:10BD20006FD1FCF7A9FCA36C4D4DC01A00282A68FE
:10BD3000B8BF4042904208D94A4B1A78012A04BF42
:10BD400002221A70FCF798FCA064FCF795FCE36CE7
:10BD50006A68C01A0028B8BF4042904208D9414BD7
:10BD60005A78012A04BF02225A70FCF785FCE0646D
:10BD7000FCF782FC236DAA68C01A0028B8BF4042B5
:10BD8000904208D9374B9A78012A04BF02229A7050
:10BD9000FCF772FC206594F8803093B394F8683116
:10BDA0007BBB304A30481D46D15C022940F00681F9
:10BDB00050F823104E1C00F000812C4A84F86431A6
:10BDC0001268C4F848212A4A1268C4F84C21A26DAE
:10BDD000C4F85021274AA1651268C4F8542194F888
:10BDE0008120C4F858210023D4F88820C4F85C21AD
:10BDF00084F88130D4F88420C4F86021012384F8C9
:10BE0000683194F87031092B06D194F85420022A35
:10BE100004BF052284F85420D4F87421002A00F0CD
:10BE2000D680092B40F0D38094F85430012B40F099
:10BE3000CE80A16D1048002350F823508D4240F071
:10BE4000C280052384F85430C1E000BF0C80FF1F7E
:10BE5000D894FF1F8894FF1F3093FF1FEF95FF1F9B
:10BE60004894FF1F9994FF1F0487FF1FE095FF1F51
:10BE7000FC95FF1FE094FF1FF087FF1F03A8FCF74E
:10BE80004DFC054600284ED0FCF760FC08B184F854
:10BE9000A36194F8A3219DF80C10531CDBB222443B
:10BEA000092B84F8A33182F8A4117FF422AF5E4AF3
:10BEB00094F8A41152780023914284F8A3317FF4BE
:10BEC00018AF5A495A5C01331644082BF6B2F9D11F
:10BED00094F8AC31B34222D1554B94F8A5211A7095
:10BEE00094F8A6215A7094F8A7219A7094F8A82182
:10BEF0009A7194F8A9215A7194F8AA211A7194F8A8
:10BF0000AB21DA70FCF7B8FB4A4B4B4A18600023B0
:10BF10001370032284F8702184F8A33196E6042379
:10BF200084F87031E5E60AAE3046FCF75AFE48B3B5
:10BF30002B46F25C01331544082BEDB2F9D19DF884
:10BF40003020AA42ECD13A4B9DF829201A709DF876
:10BF50002A205A709DF82B209A709DF82C209A71F7
:10BF60009DF82D205A719DF82E201A719DF82F20D2
:10BF7000DA70FCF781FB2F4B18602F4B00221A70F0
:10BF8000072361E694F85430013B012B3FF6B1AE34
:10BF9000A36DB3F5C05F0CD2FCF7FEFD48B1A06DF8
:10BFA0002349431CA365FCF758FF092384F870312B
:10BFB00053E6002384F854309BE6D55401332F2BED
:10BFC0007FF4F2AE1DE701339A427FF435AF0FB034
:10BFD000BDE8F08394F87001082804D840F25112AB
:10BFE000C240D207F3D4D4F86C01144DD3F8033017
:10BFF0006970B0F5C05F6B6012D20D49FCF726FF87
:10C000000B49D4F86C01FCF74CFF38B1D4F86C3113
:10C010000133C4F86C3165232B70D8E70723FBE7A5
:10C0200007232B7000230DE70C80FF1F1C88FF1FC8
:10C03000D894FF1F9094FF1F9794FF1FF495FF1F44
:10C04000704710B5074CFCF717FB2368C01AB0F512
:10C05000FA7F05D9044B0222DA60FCF70DFB206061
:10C0600010BD00BF009AFF1F00F00F40704708B5D9
:10C07000034B5878FCF738FD024B586008BD00BFF1
:10C08000D894FF1FF495FF1F7047704770477047A3
:10C09000704708B5034B3B21987801F0B7F8024B85
:10C0A000586008BDD894FF1FF495FF1F00000000E2
:10C0B000014B53F8200070472888FF1F2DE9F74FE8
:10C0C000AF4CE369C3B1AF4D2E78AEB9FCF7D4FAEB
:10C0D000AD4B1B68C01A0028E369B8BF40429842C4
:10C0E0000AD9304601F078FC012001F075FC0220ED
:10C0F00001F072FC01232B70236AC3B1A34D2E788B
:10C10000AEB9FCF7B9FAA24B1B68C01A0028236A23
:10C11000B8BF404298420AD9304601F05DFC012088
:10C1200001F05AFC022001F057FC01232B70994CBE
:10C13000FCF7A2FA237E04EB8303DB68C01A002815
:10C14000B8BF40420A2828DDFCF796FA21210746AD
:10C15000207E01F05BF894F8188004EB8805064611
:10C16000EB69C31A07EE903AEB68FB1AB8EEE77A70
:10C1700007EE903AF8EEE77AC7EE276A16EE900AD5
:10C1800003F00CFE7CA3D3E9002303F05BFE04F074
:10C19000F3F844F82800EF60EE613521207E01F0CD
:10C1A00035F810F0400905460DD0207E01F014FC52
:10C1B000237E794A0121D1540F33784AD15C012979
:10C1C00004BF0221D154207E754E06EB80131B69FB
:10C1D000002B55D0222101F019F8277E06EB87139A
:10C1E00000281B69B8BF4042984249D9E31993F827
:10C1F000283073B93421384601F008F8342140F46E
:10C200008062384600F0BEFF237E0122234483F87B
:10C21000282094F82B70DFF890B157B9F8B2FCF7EA
:10C2200014FC0BF807000137082FF7D1012384F81D
:10C230002B305C49DFF864A127274FF00008022269
:10C240005FFA88F08DE80600FCF7FFFB1BF808306A
:10C2500083429DE806002ED008F108030BF8080081
:10C2600051F82330022B1FD0032B02D0012B22D1F7
:10C2700008B31AF80730012B08BF0AF807201AE0A4
:10C28000277EE31993F82830002BC2D0342138469A
:10C2900000F0BCFF342120F48062384600F072FFC9
:10C2A000237E00222344B2E728B91AF807000128A8
:10C2B00001D10AF8073008F10108B8F1080F07F1B9
:10C2C0000107BDD1237E15F0010104EB03023CD030
:10C2D00092F8341089B9012182F83410314A1A4495
:10C2E000127E12F0010F08D002211B2211FB032342
:10C2F0002A4AD05C012808BFD154237EE218AF0738
:10C3000092F837102DD589B9012182F83710254AC6
:10C310001A44D27E12F0010F08D00E331F4A12F8D1
:10C320001310012904BF022102F8131015F0800137
:10C330003CD0237E194A0333D05C012801D102206E
:10C34000D054B9F1000F3DD033E092F8340000280A
:10C35000D3D082F83410134A1A44127E12F0020F1E
:10C36000C1E70029E2D0012182F837100D4A1A44B2
:10C37000D27E12F0020FCFE7FCA9F1D24D629040BD
:10C380000C80FF1F9794FF1F9094FF1F3093FF1F97
:10C390008894FF1F2888FF1F7093FF1F9994FF1F29
:10C3A0007893FF1F4894FF1F5488FF1FB9F1000FB7
:10C3B0001CD0237E2A4A0F33D05C012804BF022000
:10C3C000D05499B12749237E0A7842FA03F0C00776
:10C3D0000CD50120244F00FA03F33B70234F387033
:10C3E0002348007810B922EA03030B70207EC02294
:10C3F000352100F0C7FE207E06EB80131B6A0BB3CD
:10C400006B051FD4392100F001FF21210546207E54
:10C4100000F0FCFE237E06EB8316281A0028326A01
:10C42000B8BF404290420DD9184601F0D5FA237E9C
:10C43000104A0121D1541533094AD15C012904BFA6
:10C440000221D154207E00F045F8237E0133DBB277
:10C45000022B88BF0023237603B0BDE8F08F00BF16
:10C460009994FF1F5293FF1F5193FF1FD794FF1FF3
:10C470004093FF1F4B93FF1F73B5134E335C04466D
:10C480000D463BB1114B262153F8202000F07AFED7
:10C490000023335585EAE572A2EBE5722046272199
:10C4A00000F070FE0A4B0122002D1A554FF00003D8
:10C4B000D8BF0222019200931A462021204600F0A4
:10C4C0000FFE02B070BD00BFD494FF1FC894FF1FC1
:10C4D0004E93FF1F2DE9F04F352185B0044600F043
:10C4E00095FE0346C0480393A10146184FEA530B3B
:10C4F000327AD6F8048012F0400F14BF415850F839
:10C5000001A003F001051FBF0BF00109C1F1000AF2
:10C510005FFA85FBC8F1000804BF5FFA85F90BF0EC
:10C52000010B150602F03F06204613D501F074FA00
:10C53000B0FA80F77F09721E039B072A00F27B8105
:10C54000DFE812F00E000E000E000E0012011201C4
:10C550001201120101F060FA071C18BF0127EAE777
:10C56000A24D2A5D013A0E2A00F26581DFE812F041
:10C570000F001E002D003B004B00540063007200B2
:10C58000A200C400CA006301F800E101DC0134210B
:10C59000204600F03BFE05EB840301225860023E7A
:10C5A000934B96421A551BD802231AE005EB8403DD
:10C5B0005A6842F002023421204600F0E3FD514661
:10C5C0002046FFF759FF03230BE0BBF1000F00F0FB
:10C5D00032812121204600F019FE864B43F82400C9
:10C5E00004232B5527E105EB84035A6842F001022E
:10C5F0003421204600F0C6FDCAF100012046FFF7B5
:10C600003BFF0523EDE7B9F1000F00F01481204650
:10C6100001F0E2F90623E4E705EB840334215A68CC
:10C62000204622F0030200F0ADFD41462046FFF710
:10C6300023FF0723D5E7B9F1000F40F0FC804946FE
:10C640002046FFF719FFC8F100012046FFF714FF4D
:10C650000823C6E7B9F1000F00F0ED802121204644
:10C6600000F0D4FD002106462046FFF705FF614A91
:10C6700052F824309B1B42F8243005EB840334210C
:10C680005A68204622F0030200F07CFD4246272132
:10C69000204600F077FD32462D21204600F072FD45
:10C6A0000023019300931A462021204600F018FD34
:10C6B000092396E7990540F1BE802121204600F02C
:10C6C000A5FD4D4B002118602046FFF7D5FE002246
:10C6D0002D21204600F056FD00222121204600F0A9
:10C6E00051FD033E00223921204600F04BFD012E72
:10C6F00038D8C8F10001B2E0B9F1000F00F09B801A
:10C700000B236EE7B9F1000F40F095802121204600
:10C7100000F07CFD494606462046FFF7ADFE05EBDE
:10C72000840334215A68204622F0030200F02AFDD7
:10C7300042462721204600F025FD02222D2196FBAE
:10C74000F2F2204600F01EFDCDF80490CDF80090E6
:10C750004B461A462021204600F0C2FC0D2340E73C
:10C760009A0568D50E233CE7204D2A5D013A0E2A32
:10C7700061D8DFE802F008192A4354606360608BD7
:10C780009579B9DED9001A4B0122342120461A5579
:10C7900000F03CFD05EB8403062E58603FF404AF27
:10C7A000082E7FF41DAFFFE6062E05D105EB8403AE
:10C7B0005A6822F00302FCE6082E7FF400AF05EB76
:10C7C00084035A6822F00302F5E6731F012B07D891
:10C7D000BBF1000F04D0062E3FF402AF0F2300E799
:10C7E0004FB30C23FDE600BF7893FF1F6488FF1F43
:10C7F0004E93FF1F3493FF1F3C94FF1F052E05D15E
:10C8000005EB84035A6822F00302EFE6072E7FF45B
:10C81000F3AE05EB84035A6822F00302E8E6731FC7
:10C82000012B05D8B9F1000F02D0052ED6D1BBE6F9
:10C83000002F7FF4FEAE05B0BDE8F08F002FFAD1D7
:10C84000073E012E0AD905EB840334215A6822F0F1
:10C85000030242F00202204600F094FC41462046CA
:10C86000FFF70AFE0A23BCE6002FE4D1073E012EA3
:10C870007FF63FAF05EB840334215A6822F00302B0
:10C8800042F00102204600F07DFC32E7002FD2D0BA
:10C890002121204600F0BAFC05EB840318612FE744
:10C8A000002FC8D1212105EB8409204600F0AEFC01
:10C8B000D9F80420064622F003023421204600F075
:10C8C00061FC42462721204600F05CFCD9F810208C
:10C8D0002D2116442046022296FBF2F200F052FC73
:10C8E000019700973B4634E79B05A4D50E232121F1
:10C8F00020462B5500F08AFC124B00211860204680
:10C90000FFF7BAFD204600222D2100F03BFC204617
:10C910000022212100F036FC00223921204605B0FA
:10C92000BDE8F04F00F02EBC00212046FFF7A4FD2B
:10C9300018E705EB840334215A68204600F022FCF6
:10C9400000234EE63C94FF1F024B1A5C0AB90122F9
:10C950001A5470476488FF1F024B1A5C0AB10F22F9
:10C960001A5470476488FF1F014B185C704700BF62
:10C970006488FF1F0C4A116940F273234B434FF642
:10C98000FF71B3FBF1F36E2B06D9084B4FF48021F6
:10C9900059605723136070474F2B9EBF034B4FF4D2
:10C9A00080219960F5E700BF00B0034080F00F40A0
:10C9B0001B4B1A6802F01F02072A2ED8DFE802F08C
:10C9C000040B2D11171D23291A69164992B20A80EA
:10C9D00041221A6070471A69124992B24A80432272
:10C9E000F7E71A690F4992B2CA804422F1E71A693F
:10C9F0000C4992B20A814522EBE71A69094992B2C1
:10CA00004A814622E5E71A69064992B28A8147229D
:10CA1000DFE71A69034992B2CA814022D9E700BF11
:10CA200000B00B408088FF1F38B541F23001114B38
:10CA30005A5842F000625A5041F23C0100245A58C0
:10CA400042F000625A5003F5E8230C2540229D6015
:10CA50004920DC605C621A6001F092F8064B5722B4
:10CA60009D602720DC605C621A60BDE8384001F000
:10CA700087B800BF0070044000B003400B2829D8DD
:10CA8000DFE800F0060A0D102828282813281E23A6
:10CA9000114B188980B270470F4B5889FAE70E4B3B
:10CAA0009889F7E70C4BD889F4E70B4B588883B289
:10CAB00040F2732058434FF6FF7390FBF3F070473A
:10CAC000054BD88883B28E20F4E7034B188883B2D5
:10CAD0004220EFE7002070478088FF1F30B52E4DC1
:10CAE00041F23C042B5943F010032B512B4B4FF4D4
:10CAF00000741C636FF4F8755C63A3F51433A4F140
:10CB00003E542C441C604FF400545C60244C1C6068
:10CB10001C68E401FCD50138072834D8DFE800F0B0
:10CB2000312F2D2B293327041E4858601E4B00201F
:10CB300058631E4818601E484FF0806400EA814523
:10CB4000C3F88040C3F88450FAB100EA8240C3F8C9
:10CB50009040C3F894004FF08460C3F8A000C3F87D
:10CB6000A410AAB1C3F8B000C3F8B42030BD114876
:10CB7000DBE71148D9E71148D7E71148D5E7114855
:10CB8000D3E71148D1E71148CFE7C3F89020E2E797
:10CB9000C3F8B02030BD00BF0070044000900440D6
:10CBA0000F0080508720FE01004002400F008000EF
:10CBB0000000FC1F8720FE038720FE0F8720FE1346
:10CBC0008720FE278720FE638720FEC78720FE0779
:10CBD000384AD2F88030C3F30363022B5FD0D2F817
:10CBE0009030C3F30363022B5BD0D2F8A030C3F3C1
:10CBF0000363022B06D0D2F8B030C3F30363022BD9
:10CC000056D103231B0103F1402202F50032D2F872
:10CC10008010C1F303410170D2F8801011F480112B
:10CC200018BF01218170D2F8801011F4001118BFD3
:10CC3000012141704178B1BBD2F88410C1F38A411F
:10CC400003F1402303F500334160D3F88810090E47
:10CC50000172D3F88810090C4172D3F88810090AC0
:10CC60008172D3F88810C172D3F88C10090E017349
:10CC7000D3F88C10090C4173D3F88C10090A817316
:10CC8000D3F88C30C373D2F880309B024CBF4FF086
:10CC900084634FF08063C2F8803001207047002326
:10CCA000B0E70123AEE7D2F8841021F06041C7E776
:10CCB0000020704700400240184AD2F87031C3F398
:10CCC00003630C2B10B527D04478436804B3C3F337
:10CCD0001103C2F874318368104A1BBAC2F8783164
:10CCE000C3681BBAC2F87C318378002C14BF4FF0A4
:10CCF00042624FF040620BB142F4801203781B0491
:10CD000003F470231343054A0120C2F8703110BDAB
:10CD1000034901EA8343DCE7002010BD00400240E4
:10CD20000000FC1F0B4B4FF00062C3F870214FF462
:10CD30008022C3F87421084AC3F878216FF4847103
:10CD4000A2F166320A44C3F87C21044AC3F8702178
:10CD5000704700BF00400240785634120000080CB3
:10CD600010B53A4BDA7842F00202DA70384A10789D
:10CD7000C0B20228114641D0032835D0012832D153
:10CD8000546891688C4215D2D978C90707D4516884
:10CD9000D0684C1C5460425CD2B21A7110BD9978B4
:10CDA00001F0DF019970997801F0EF01997010742A
:10CDB000002317E0517C01F0FF0049B9997801F098
:10CDC000DF019970997801F0EF019970107010BD32
:10CDD000997841F004019970917CC9B219710023CE
:10CDE00053740323137010BD997801F0EF0199700B
:10CDF0001B795169DBB20B700223F3E79469D069A8
:10CE000084421DD2D2698869121A012A05D19A7802
:10CE100002F0DF029A7000230B70CB698A699B1ABB
:10CE2000022B9FBF094A937843F0080393708A69E5
:10CE30004869531C8B61054B1B79DBB2835410BDD1
:10CE4000997801F0DF019970B2E700BF00700640E9
:10CE50009488FF1F41F234020A498B5843F0800343
:10CE60008B50094B4FF418729A62DA6203F5E03383
:10CE70001B225A70C0229A7000225A71192000F0A9
:10CE80007FBE00BF0070044000B0044010B5104BDE
:10CE900000241C745C749A6001225C601A700D4A54
:10CEA000D960917801F0F7019170917841F010010B
:10CEB0009170917800F0FE0041F0200191701071A6
:10CEC0001A78002AFCD1187CB0FA80F0400910BD15
:10CED0009488FF1F0070064010B5104B00241C748E
:10CEE0005C74DA6103229C611A700D4A5961917871
:10CEF00001F0F7019170917841F0100191709178F3
:10CF000040F0010041F02001917010711A78002A60
:10CF1000FCD1187CB0FA80F0400910BD9488FF1F46
:10CF20000070064070B5144C002563610126049B17
:10CF300025746674A2606560E36140EA0603A5613A
:10CF4000A3740E4BE16026709A7802F0F7029A7093
:10CF50009A7842F010029A709A7800F0FE0042F03F
:10CF600020029A7018712378002BFCD1207CB0FA33
:10CF700080F0400970BD00BF9488FF1F007006401C
:10CF800010B50024E0B24FF480323A21013400F0B1
:10CF9000F9F8032CF6D110BD2DE9F7434A4D05EB06
:10CFA00080150446EB690BB16E8B96B9382120468B
:10CFB00000F02CF9382120F48062204600F0E2F8DD
:10CFC0004FF480323A21204603B0BDE8F04300F030
:10CFD000D9B800F0BAFAC0F1080006FA00F002F081
:10CFE000CBFEED69064685EAE570A0EBE5700F46DD
:10CFF00002F0C2FE02460B463046394603F04CF8BA
:10D000000022324B8046894602F01CFF0F4606463E
:10D0100047EC106B684603F09BFA0022002351ECAA
:10D02000100B03F077F9A0B13046394603F0A4F9AC
:10D03000002D06464FF03801B8BF4642204600F0AA
:10D04000E5F8382120F48062204600F09BF8324653
:10D05000B8E7684649EC108B03F07AFA002D57ECDC
:10D06000106BDDE9000118DD03F086F914A3D3E9A4
:10D07000002305043946304602F0E4FE03F07CF953
:10D0800005433821204600F0C1F8382140F4806281
:10D09000204600F077F82A4694E703F06DF908A3DC
:10D0A000D3E90023C5433946304602F0CBFE03F0F6
:10D0B00063F9C0F51C502D041030E1E7AFF3008098
:10D0C000000000000088C3407893FF1F0000F0407C
:10D0D000392100F09BB80A46392100F053B800BF4F
:10D0E0002DE9F74F01F07F05352D1C460746934685
:10D0F0009DF830909DF83480204E4FEA022314D1E1
:10D100001C4349EA042448EA04249F3024F473644D
:10D1100024F00304E40456F82030E40C23EA040469
:10D1200046F8204003B0BDE8F08F154A019332F86D
:10D1300010A041F0800100225046FBF7BDFD002207
:10D1400059465046FBF7B8FD214600225046FBF7F2
:10D15000B3FD002249465046FBF7AEFD0122414691
:10D160005046FBF7A9FD019B1C4349EA042405EB4B
:10D170004500384448EA0424D2E700BFB488FF1FC2
:10D18000D80901002DE9F04101F07F05352D064653
:10D190001446DFF874800FD100F19F0522F4736408
:10D1A00024F0030458F82530E404E40C23EA0403D3
:10D1B00048F82530BDE8F081124B33F8107000229A
:10D1C00041F080013846FBF777FD0022210E3846FA
:10D1D000FBF772FD05EB45050022C4F30741384615
:10D1E000FBF76AFD35440022C4F307213846FBF7FC
:10D1F00063FD0122E1B23846FBF75EFD48F82540A9
:10D20000BDE8F081D8090100B488FF1FF8B5324BA2
:10D2100001F07F055A190646127B002A54D033F8D4
:10D220001070002229463846FBF746FD00221146C1
:10D230003846FBF741FD002211463846FBF73CFD1E
:10D24000002211463846FBF737FD012200213846FF
:10D25000FBF732FD002211463846FBF72DFD002278
:10D2600011463846FBF728FD0022114604023846D5
:10D27000FBF722FD0022114604433846FBF71CFD54
:10D2800024020443012200213846FBF715FD240245
:10D29000352D40EA04000ED1104A06F19F0552F8E0
:10D2A000253023F4736323F00303DB04DB0C184302
:10D2B00042F82500F8BD222D01D0422D0AD10302EB
:10D2C00008D540F07F40F8BD05EB45050544034B0C
:10D2D00053F82500F8BD00BFD8090100B488FF1F2E
:10D2E00070B50B4C2218054692F800260E465AB926
:10D2F0006C21FFF78BFF06F00F0320F00F021A439B
:10D300006C212846FFF73EFF631983F8036670BD62
:10D31000B488FF1F38B50C466C210546FFF776FF31
:10D32000240104F0700420F07002224328466C218E
:10D33000BDE83840FFF726BF38B50C466C210546DE
:10D34000FFF764FFE40304F4C03420F4C032224346
:10D3500028466C21BDE83840FFF714BF38B50C46AD
:10D360006C210546FFF752FF240504F4700420F4F5
:10D370007002224328466C21BDE83840FFF702BF07
:10D3800038B50C466C210546FFF740FF240604F033
:10D39000706420F07062224328466C21BDE838405A
:10D3A000FFF7F0BE38B50D466C210446FFF72EFF9F
:10D3B0003DB140F0804220466C21BDE83840FFF787
:10D3C000E1BE20F08042F6E738B50D466C210446F8
:10D3D000FFF71CFF3DB140F4002220466C21BDE860
:10D3E0003840FFF7CFBE20F40022F6E738B50D46EF
:10D3F0006C210446FFF70AFF3DB140F4802220462D
:10D400006C21BDE83840FFF7BDBE20F48022F6E76E
:10D4100038B50D466C210446FFF7F8FE3DB140F4E7
:10D42000804220466C21BDE83840FFF7ABBE20F4B7
:10D430008042F6E738B50D466C210446FFF7E6FE5C
:10D440003DB140F4005220466C21BDE83840FFF762
:10D4500099BE20F40052F6E738B50D466C2104461B
:10D46000FFF7D4FE3DB140F4805220466C21BDE868
:10D470003840FFF787BE20F48052F6E738B50C46F7
:10D480006C210546FFF7C2FE230748BF20F070005D
:10D490004FEA04124CBF40F4006020F4076002F031
:10D4A000700202436C212846BDE83840FFF76ABE8F
:10D4B00038B50C466C210546FFF7A8FEE40104F4DC
:10D4C000F06420F4F062224328466C21BDE8384025
:10D4D000FFF758BEFFF7ECBF38B50D466C21044688
:10D4E000FFF794FE3DB140F4003220466C21BDE8C8
:10D4F0003840FFF747BE20F40032F6E708B5074B87
:10D50000034493F800262AB96C21FFF77FFE00F050
:10D510000F0008BD93F8030608BD00BFB488FF1FC5
:10D5200008B56C21FFF772FEC0F3021008BD08B504
:10D530006C21FFF76BFEC0F3C13008BD08B56C214C
:10D54000FFF764FEC0F3035008BD08B56C21FFF778
:10D550005DFEC0F3036008BD08B56C21FFF756FE01
:10D56000C0F3807008BD08B56C21FFF74FFEC0F313
:10D57000C04008BD08B56C21FFF748FEC0F38040ED
:10D5800008BD08B56C21FFF741FEC0F3803008BD2F
:10D5900008B56C21FFF73AFEC0F3403008BD08B56E
:10D5A0006C21FFF733FEC0F3003008BD08B56C21D5
:10D5B000FFF72CFEC0F30213020548BF43F0080337
:10D5C000184608BD08B56C21FFF720FEC0F3C31054
:10D5D00008BDFFF7F7BF08B56C21FFF717FEC0F3D2
:10D5E000404008BD38B50C466D210546FFF70EFEDC
:10D5F000640104F0600420F06002224328466D219B
:10D60000BDE83840FFF7BEBD38B50C466D21054674
:10D61000FFF7FCFD640304F4C04420F4C04222433D
:10D6200028466D21BDE83840FFF7ACBD38B50C4643
:10D630006D210546FFF7EAFD240204F4706420F42E
:10D640007062224328466D21BDE83840FFF79ABD3D
:10D6500038B50C466D210546FFF7D8FD04F00F04E0
:10D6600020F00F02224328466D21BDE83840FFF725
:10D6700089BD38B50D466D210446FFF7C7FD20F47E
:10D680007F0040EA05426D212046BDE83840FFF7A3
:10D6900079BD38B50D466D210446FFF7B7FD3DB1A4
:10D6A00040F4004220466D21BDE83840FFF76ABDD6
:10D6B00020F40042F6E738B50D466D210446FFF729
:10D6C000A5FD3DB140F0807220466D21BDE8384097
:10D6D000FFF758BD20F08072F6E708B56D21FFF71F
:10D6E00095FDC0F3411008BD08B56D21FFF78EFD13
:10D6F000C0F3413008BD08B56D21FFF787FDC0F3C9
:10D70000032008BD08B56D21FFF780FD00F00F0074
:10D7100008BD08B56D21FFF779FD0314D8B21B06CB
:10D7200048BF60F0FF0008BD08B56D21FFF76EFD32
:10D73000C0F3C03008BD08B56D21FFF767FDC0F329
:10D74000006008BD38B50C4670210546FFF75EFD48
:10D7500004F0030420F4401242EA045228467021E7
:10D76000BDE83840FFF70EBD38B50D4670210446C0
:10D77000FFF74CFD3DB140F4002220467021BDE88A
:10D780003840FFF7FFBC20F40022F6E738B50D461D
:10D7900070210446FFF73AFD3DB140F48022204657
:10D7A0007021BDE83840FFF7EDBC20F48022F6E799
:10D7B00038B50C4670210546FFF728FD04F0030438
:10D7C00020F4403242EA044228467021BDE8384045
:10D7D000FFF7D8BC38B50D4670210446FFF716FD9B
:10D7E00020F47F4040EA052270212046BDE8384001
:10D7F000FFF7C8BC38B50D4670210446FFF706FD9B
:10D8000020F0FF0045EA000270212046BDE83840C4
:10D81000FFF7B8BC08B57021FFF7F8FCC0F3015062
:10D8200008BD08B57021FFF7F1FCC0F3C04008BD8A
:10D8300008B57021FFF7EAFCC0F3804008BD08B5C9
:10D840007021FFF7E3FCC0F3014008BD08B570216B
:10D85000FFF7DCFCC0F3072008BD08B57021FFF717
:10D86000D5FCC0B208BD70B50E466F2115461C46EA
:10D87000FFF7CCFC16B1C0F34923336015B1C0F3F8
:10D8800004432B700CB1000E207070BD2DE9F743DE
:10D89000FAF7F2FE0446FAF7EFFE001B0028B8BFC5
:10D8A00040420928F7DD384F0025A946A7F10308B3
:10D8B000ECB2002211462046FFF764FC02225523F9
:10D8C0008DE80C006C21012300222046FFF708FCA4
:10D8D00001260F238DE8480000220723102120464F
:10D8E000FFF7FEFB294A70212046FFF74BFC20463C
:10D8F000FFF704FE05F80890785500222021204605
:10D90000FFF740FC00222D212046FFF73BFC0022C0
:10D9100021212046FFF736FC324623212046FFF71F
:10D9200031FCDC2224212046FFF72CFC46F6DB02EA
:10D9300025212046FFF726FC40F2B712262120467B
:10D94000FFF720FC4DF2B71227212046FFF71AFC03
:10D9500040F2B71228212046FFF714FCDC222A21CE
:10D960002046FFF70FFC0A222B212046FFF70AFC76
:10D970003544074A14212046FFF704FC032D97D1B4
:10D9800003B0BDE8F08300BFB78EFF1F8004050021
:10D99000FFFF0F0038B5074C044494F8001641B956
:10D9A00094F80356FFF79CFC012384F8003684F8B2
:10D9B000035638BDB488FF1F064B034493F8002676
:10D9C00032B1002293F8031683F80026FFF788BCD3
:10D9D000704700BFB488FF1F0D4B37B501251D549C
:10D9E0000C4BC4B21D54002220462721FFF7CAFB6E
:10D9F00020464FF6FF722621FFF7C4FB0023019556
:10DA000000931A4620212046FFF76AFB03B030BD81
:10DA10004E93FF1FD494FF1F012809D003D302287F
:10DA20000BD000207047074B1869C0F38050704737
:10DA3000044B1869C0F340507047024B1869C0F39B
:10DA40000050704740F00F40002808B50FDB02F08F
:10DA500093F90DA3D3E9002302F01EFB41EC100B58
:10DA600002F0F2FE51EC100B02F086FC08BD02F051
:10DA700083F905A3D3E9002302F00EFB41EC100B60
:10DA800002F04EFEEEE700BF34F7FFFF7F84EE3F6B
:10DA900008B502F071F908A3D3E9002302F0FCFAFB
:10DAA00041EC100B02F0D0FE51EC100B02F064FCC4
:10DAB00008BD00BFAFF30080EB1100A2941A5D40D7
:10DAC000002808B50FDB02F057F90DA3D3E90023B6
:10DAD00002F0B8F941EC100B02F022FE51EC100BF1
:10DAE00002F04AFC08BD02F047F905A3D3E9002380
:10DAF00002F0A8F941EC100B02F0A6FEEEE700BF21
:10DB000034F7FFFF7F84EE3F07EE900AF8EEE77AE6
:10DB100008B517EE900A02F041F907A3D3E90023F4
:10DB200002F090F941EC100B02F0FAFD51EC100BF1
:10DB300002F022FC08BD00BFEB1100A2941A5D4068
:10DB4000704700BFFEE74FF0E0210B4A0B4BC1F8D6
:10DB5000083D4CF22053D3814DF62813D38113880E
:10DB600023F001031B041B0C1380D1F8883D43F400
:10DB70007003C1F8883D7047002005400080000018
:10DB8000802800F01F014FF001030F4A04DD8B4095
:10DB9000C2F88C31D3607047402804DD8B40C2F856
:10DBA000883193607047202804DD8B40C2F88431AF
:10DBB00053607047404200F01F0058BF41428B4005
:10DBC000C2F880311360704700E100E0802800F067
:10DBD0001F024FF001030D4903DD9340C1F88C3063
:10DBE0007047402803DD9340C1F8883070472028F3
:10DBF00003DD9340C1F884307047404200F01F00BD
:10DC000058BF42429340C1F88030704700E100E0C5
:10DC1000074B1A78D2B2012A02D1222903D15A70B5
:10DC200001225A7070472129FAD10022F7E700BF7C
:10DC3000BA8EFF1F70B5154611B91B4B197070BD18
:10DC4000022903D1184B01221A7070BD04291AD180
:10DC5000154B5B78012B25D19488402C28BF40249C
:10DC600000235E1CDBB2A34207D300231A46022125
:10DC70001846BDE8704000F047BF2A68D05C00F04D
:10DC8000C3F83346EDE7032906D1074A5378012B41
:10DC900008D100239370E9E7052901BF024B002258
:10DCA0001A705A7070BD00BFBA8EFF1F10B50446BF
:10DCB000204600F0C1F80028FAD110BD704738B5F1
:10DCC0000A4C012502460B4600202946A57000F0AB
:10DCD000F5FA224618B10023A370122038BD9378BC
:10DCE00003F0FF00002BFAD138BD00BFBA8EFF1F32
:10DCF000F8B506460F4600F0F4FC0E4B1A78012AE0
:10DD000016D15B78012B13D100F000F988B1002502
:10DD1000ECB2A74205D821463046BDE8F840FFF7EF
:10DD2000CEBF301900F0D6F801350028F0D0F2E768
:10DD30000C20F8BDBA8EFF1F08B540210248FFF73E
:10DD4000D7FF00F095F808BDBD8EFF1F38B505461A
:10DD500000F0A8F80B28044609D140210548FFF738
:10DD6000C7FF28B92846BDE8384000F09BB800241A
:10DD7000204638BDFD8EFF1F70B50C46461E00259F
:10DD80000CB9284670BD16F8010FFFF7DFFF013C04
:10DD9000002818BF0B25A4B2F2E738B5451E0024B1
:10DDA00015F8010F08B9204638BDFFF7CFFF00284E
:10DDB00018BF0B24F4E707B501230022009306499E
:10DDC000064B104600F020FA002814BF1B2000204C
:10DDD00003B05DF804FB00BF35DC000011DC00007F
:10DDE00038B50C46054600F097F8A0420AD32C44FB
:10DDF0000020A54207D000B138BD15F8010B00F096
:10DE000051F8F6E70B2038BD10B50A4A11784029C1
:10DE10000ED05378D4180133DBB2402BA07001F13F
:10DE200001014FF00000117014BF5370507010BD0D
:10DE30000B2010BD3D8FFF1F10B50C4A117891B11A
:10DE400092F84230D4180133DBB2A4780470402B2E
:10DE50004FF0000001F1FF31117014BF82F8423021
:10DE600082F8420010BD0A2010BD00BF3D8FFF1F89
:10DE7000014B1878704700BF3D8FFF1F024B187889
:10DE8000C0F14000C0B270473D8FFF1F034B00221E
:10DE90005A7083F842201A70704700BF3D8FFF1FF1
:10DEA000FFF7F4BF10B50A4A117840290ED0537815
:10DEB000D4180133DBB2402BA07001F101014FF007
:10DEC0000000117014BF5370507010BD0B2010BDB6
:10DED000808FFF1F10B50C4A117891B192F8423033
:10DEE000D4180133DBB2A4780470402B4FF000004B
:10DEF00001F1FF31117014BF82F8423082F8420004
:10DF000010BD0A2010BD00BF808FFF1F014B187885
:10DF1000704700BF808FFF1F024B1878C0F1400090
:10DF2000C0B27047808FFF1F034B00225A7083F8E6
:10DF300042201A70704700BF808FFF1FFFF7F4BFA9
:10DF400070B50546007801F093F902780023D9B244
:10DF5000914207D25C1C03EB830303445E786B7829
:10DF60009E4227D1174C2B7A342202FB0142D678ED
:10DF700013B334234B43E218907886420CD000F060
:10DF8000030204330C2010FB02302118205C0B89A3
:10DF90004A68497800F090FBD4F89C3083B12A4657
:10DFA000287812F8081F00290CBF03210521BDE8BD
:10DFB000704018472346CAE7937801339370D8E737
:10DFC00070BD00BFC48FFF1F2DE9F04F85B00D4617
:10DFD00090468DF80F0001F04BF9022D064647D10F
:10DFE000077800235C1CDBB2BB4210DB4FF000095A
:10DFF000DFF8B0B0CA465FFA89F4A74212DC284BBA
:10E00000D3F89C30002B45D105B0BDE8F08F03EB71
:10E01000830333440DF10F00DA78597801F0E2F907
:10E020002346DFE704EB84043444E378A288617874
:10E03000CDF804A0A07800900DF10F0001F0B0F928
:10E04000A378032B05D15A4661789DF80F0001F0A3
:10E0500031FA6178E37841F0100141EAC3110022FE
:10E06000C9B20DF10F0001F0EDF909F10109C2E7A4
:10E07000002DC4D10A490378342000FB03138A1C05
:10E080003633294634329A42B9D002F8341C02F8A9
:10E09000331CF7E7424629469DF80F009847B3E73F
:10E0A000C48FFF1F41DF0000F0B40C7804F060045F
:10E0B000202C1D4632D14C78042C1DD00AD8012CBE
:10E0C00004D003D3022C20D0032C12D000202880AF
:10E0D000F0BC7047212C1BD004D8202CF6D1F0BC0A
:10E0E00000F040B9222C16D0232CEFD1F0BC00F068
:10E0F00049B9F0BC00F049B902241C80146800251D
:10E1000025701468671C17606570F0BC00F056B984
:10E11000F0BC00F01FB9F0BC00F076B9402C06D17D
:10E12000044CD4F8A04014B1A446F0BC6047CD2004
:10E13000CEE700BFC48FFF1F73B50446007801F01F
:10E1400097F863680093A27A637A43EA0223ADF8F2
:10E15000043002780023D9B2914207D25D1C03EB50
:10E16000830303445E7863789E4225D1174D237A5A
:10E17000342202FB0152D67803B334234B43EA180E
:10E18000907886420CD000F0030204330C2010FB80
:10E1900002302918285C0B894A68497800F08CFA0B
:10E1A000D5F89C3033B1227A20785AB104F10802B4
:10E1B0000521984702B070BD2B46CCE79378013318
:10E1C0009370DAE76A460321F3E700BFC48FFF1FAD
:10E1D00007B543680093437A817A43EA0123ADF897
:10E1E0000430084BD3F89C3002462BB1017A0078FA
:10E1F00029B108320521984703B05DF804FB6A464F
:10E200000421F8E7C48FFF1F2DE9F84305460F46A8
:10E210001646984601F02CF802789DF8203001321D
:10E220008146D2B20021284601F09EF80446E8B9A2
:10E23000164A1749284600F086F999F80000154B50
:10E24000342200FB022209F101011A4499463433B9
:10E25000934201F105010CD14146284600F074F8C3
:10E26000044618B9C9F89C70C9F8A0602046BDE8FA
:10E27000F88311F8050C03F8340C11F8040C03F8BA
:10E28000330C03F8324C03F8314CE0E7A9E000000E
:10E29000C9DF0000C48FFF1F08B5074B0022C3F879
:10E2A0009C20C3F8A02000F0A1F918B9BDE80840EF
:10E2B00001F06EB808BD00BFC48FFF1F2DE9F0410B
:10E2C000984605460E46174600F0D2FF0478002314
:10E2D000D9B2A14207D2013303EB8302024412F800
:10E2E000042CB242F4D1174C34234B43E218D078BB
:10E2F00092F802E0A0EB0E01C9B2042902D1C120BC
:10E30000BDE8F08100F003010130C0B24FF00C0C09
:10E310000CFB0133D070A0EB0E001C44C0B20128EE
:10E3200025716671A760A4F80C8007D143463A4670
:10E3300031462846BDE8F04100F0BEB90020BDE8F6
:10E34000F08100BFC48FFF1F014B00201960704790
:10E350006890FF1F024B0979197100F08DBF00BF53
:10E360006890FF1F13B5002402AA1C80044B42F8DA
:10E37000041D0979197100F08DFF02B010BD00BFB6
:10E380006890FF1F00201880704730B40C460221AF
:10E39000198021796488084D012C297102D130BC83
:10E3A00000F08EBF022C02D130BC00F095BF0020DF
:10E3B000188030BC704700BF6890FF1F30B40C4617
:10E3C0000221198021796488074D012C297102D11D
:10E3D00030BC00F08DBF022C02D130BC00F09ABFDF
:10E3E0000020188030BC70476890FF1F044B054A1E
:10E3F00019795B791171137203210A23FFF75EBF4C
:10E400006890FF1F4C80FF1FF8B500271F808B7896
:10E410000B4CA371C3F340035A0063F3000206469A
:10E420006271FFF7E3FF256845B1A37913F002029B
:10E430001ABF3A46222121213046A8470020F8BDC4
:10E440006890FF1F034B00F108021B68007805214C
:10E45000184700BF7090FF1F70B5094D04462A1D74
:10E46000012100F0D7FF80220121204600F0EAFFC1
:10E470002B68207800220A21BDE87040184700BFB1
:10E480007090FF1F37B501210DF10702044600F01F
:10E49000C1FF9DF80730074D802B04D12A79012157
:10E4A000204600F0CFFF2B68207800220B219847F0
:10E4B00003B030BD7090FF1F436805215A7800F00B
:10E4C000C1BF73B50122002405460126002100F0DA
:10E4D00089FF334621468DE850001022284600F07F
:10E4E0005FFF22462146284600F07CFF2346214656
:10E4F0008DE850001022284600F052FF31460222DB
:10E50000284600F09FFF32460621284600F09AFF79
:10E5100022469021284600F095FF044B28781B687E
:10E520002246214602B0BDE8704018477090FF1F98
:10E5300042783AB9C178C90141F0100101F0900167
:10E5400000F080BF704773B50C468DF8070001F0EE
:10E550000DFA1F4D2C600446002836D11D4A9DF847
:10E560000700102100F0A6FF1B4A044612219DF867
:10E57000070000F09FFF194A044314219DF807008B
:10E5800000F098FFE4B20443154A9DF807001321F8
:10E5900000F090FFE4B20443124A9DF807001721EF
:10E5A00000F088FF02AEE4B204430F4A16F8010DF2
:10E5B000162100F07FFFE4B204430322012130461C
:10E5C00000F040FF0323E4B22B71204602B070BD7F
:10E5D0007090FF1FC3E40000B9E4000059E400009C
:10E5E00085E4000031E5000045E4000037B502ADE8
:10E5F000174B05F8010D0022102128461A6000F083
:10E600005BFF12210446284600F056FF1421044304
:10E61000284600F051FFE4B204431321284600F0DD
:10E620004BFFE4B204431721284600F045FFE4B253
:10E6300004431621284600F03FFFE4B2204310F0C7
:10E64000FF0003D19DF8070001F09CF903B030BD35
:10E650007090FF1F1FB501218DF807000DF10E020C
:10E660000DF1070000F0D6FE0DF10F0206210DF1AD
:10E67000070000F0CFFE9DF80E30802B18D19DF8DA
:10E680000F309B0714D59DF8070000F0EFFD01281F
:10E6900004460DD172B60DF1070000F029FB0022EF
:10E6A00021460DF107008DF80E2000F0CBFE62B67A
:10E6B0009DF80E0004B010BD73B50C4615461E46FD
:10E6C0008DF80700FFF7C6FF802808D033462A469A
:10E6D00021460DF1070000F0A7FA02B070BD00203E
:10E6E000FBE77047062812D880000129C0B201D18B
:10E6F0000230C0B2074AC0F34703122101FB0323D3
:10E700001A884FF6FF739A4208BFFF207047FF2018
:10E71000704700BF7890FF1F2DE9F041314C324D1A
:10E72000324E4FF0000884F800814FF4107285F8E3
:10E7300040020F462846FF2101F0BCFE4FF48062E4
:10E7400041463046C5F8446201F0B4FE94F80C31FD
:10E7500043F0800384F80C3194F80C311B06FBD491
:10E76000234BFF221A7094F80C3143F0400384F8D5
:10E770000C31204B196897B341F000411960194BD7
:10E78000310AC6F3074201F0FE0183F89C1083F8BA
:10E79000B020320E83F8B420174AC5F84822102260
:10E7A00083F80821012283F89420BF2283F8802077
:10E7B00093F8002102F07F0283F8002193F884206F
:10E7C00042F0010283F8842093F8842042F0100282
:10E7D00083F8842084221A770020BDE8F08121F09C
:10E7E0000041CBE7002007407890FF1F009CFF1FEF
:10E7F0005680FF1F00700440009EFF1F0D4B93F8D2
:10E800000C2102F0BF0283F80C21BF2283F8802084
:10E8100093F8842002F0FE0283F8842093F8942079
:10E8200002F0FE0283F894201A7F02F07B021A772E
:10E830000020704700200740F7B5082304248DE826
:10E840001800B1F803300D788878B3F5007F81BFE8
:10E850000023CB7002230B71062D71D8AB00DCB204
:10E86000012804BF0234E4B24FEA540E354C12279B
:10E8700007FB0E474FF6FF76B7F800C0B4455FD1EF
:10E880004E78032E5CD801285AD897F80FC0BCF1F7
:10E89000FF0F04BF4FF0000C87F80FC0B1F803C0A2
:10E8A000122101FB0EFE04EB0E0743EA4003BA738C
:10E8B000FA7B7E7402F0010213435BB2D4F8482263
:10E8C000C7F80220D9B2F9733874D4F8447224F826
:10E8D0000EC01BB207EBC30E81F00101CEF804207D
:10E8E000AEF802C04FF0080E07F833E007EBC10E98
:10E8F000CEF80420AEF802C012FA8CF24FF0480EA7
:10E9000007F831E0C4F8482228B917F8332062F03C
:10E910007F0207F8332002AA02EB80002DB20A49D9
:10E9200050F8082C11F82530012E0CBF164642F085
:10E9300001063343DBB201F82530002003B0F0BDFF
:10E940009520FBE77890FF1FC0200740084610B5D0
:10E950001146FFF7C7FEFF281DD0104B1221C0F350
:10E96000470001FB0030D3F84422C37B1CB283F084
:10E97000010312F8341001F07F0102F8341012F88C
:10E98000331001F07F0102F833104FF0FF33837230
:10E99000C372002010BDC42010BD00BF7890FF1FBF
:10E9A00073B50C468DF80700114620461646FFF752
:10E9B00099FEFF28054620D0214632460DF107007A
:10E9C000FFF7C4FFC5F3470312210D4D59436B18E0
:10E9D000D5F848221888121AC5F8482224B2094AE4
:10E9E000002002F824004FF0FF326A549A705A70E7
:10E9F000DA701A715A7102B070BD9620FBE700BF41
:10EA00007890FF1FC02007402DE9F0410E46804658
:10EA1000114630461746FFF765FE0C4DC0F3470020
:10EA2000122303FB0050C47BFF2C0DD03A46314625
:10EA30004046FFF78BFF24B2D5F8442212F8343059
:10EA400063F07B0302F83430BDE8F0817890FF1F5B
:10EA500010B5084600211446FFF744FE084AC0F3EB
:10EA60004700122101FB0020D2F84432C27B03EBA5
:10EA7000C2035A68136823605368636010BD00BF07
:10EA80007890FF1F10B50C4620461146FFF72AFE6E
:10EA9000FF281AD024B2104B13F82430DBB213F045
:10EAA0000C0F12D09B0712D40C4BD3F8443213F83E
:10EAB0003020D2090DD180F00100C0B213F83030FF
:10EAC000DB0914BF0320002010BD052010BD01206C
:10EAD00010BD032010BD00BFC02007407890FF1F6D
:10EAE00008B5FFF7FFFD074A1223C0F3470003FBF9
:10EAF0000020C37BFF2B1EBFD2F84422002102F866
:10EB0000331008BD7890FF1F2DE9F0410846002121
:10EB100090461F46FFF7E6FD2249C0F34700122446
:10EB200004FB0014E57BFF2D39D022884FF6FF70DF
:10EB300093B2834233D0D1F8441285F0010011F929
:10EB4000300000282BDB2EB287B901EBC603384614
:10EB50005A80D4F802205A6011F8352002F04002A1
:10EB600062F0770201F83620BDE8F08101EBC602C1
:10EB7000BB424FF0000028BF3B466781C4F80680C7
:10EB8000207360735380C2F8048011F8353003F0AD
:10EB9000400363F0770301F83630BDE8F08194203C
:10EBA000BDE8F0817890FF1F2DE9F0410C46064644
:10EBB000114620461546FFF795FD194BC0F3470057
:10EBC000122202FB003090F80FE0BEF1FF0F24D0BC
:10EBD00027B2144A6CB1407C012D0CBF14211821BE
:10EBE000012818BF41F0010112F82700014302F883
:10EBF000271012F827106FF3410102F82710D3F8FD
:10EC00004432002203F83E203DB92B462A462146D5
:10EC10003046BDE8F041FFF777BFBDE8F08100BFA7
:10EC20007890FF1FC02007402DE9F0410C46204698
:10EC3000012117469846FFF755FDFF2836D01C4B9B
:10EC4000C0F34700122202FB0030D3F8446290F870
:10EC50000FE016F93E30002B28DB23B2154A12F8DC
:10EC6000235015F0020521D10188C0F806701FFA63
:10EC700088F242818A42D8BF11460FFA8EF206EB23
:10EC8000C2030573457359805F602CB9C82306F829
:10EC900032302046BDE8F08116F83E3003F04003E4
:10ECA00063F0770306F832302C46F2E79324F0E75E
:10ECB0007890FF1FC0200740034B044883F898104A
:10ECC0000122114600F0BEBB00200740B892FF1F92
:10ECD000054B0648002283F89420802283F80C21FB
:10ECE0000121FF2200F0AEBB00200740B892FF1FB9
:10ECF00038B51A4C94F8002102F07F0284F8002104
:10ED000094F80C2102F0DF0284F80C2194F88020A2
:10ED100042F0200284F8802094F8842002F0DF0280
:10ED200084F8842094F8942002F0DF0284F8942080
:10ED300094F8942042F0040284F8942044F620656C
:10ED4000013DADB200F0BCFE002DF9D194F8943035
:10ED500003F0FB0384F8943038BD00BF0020074067
:10ED60002DE9F04FD84DD94C95F8807095F8843046
:10ED700095F8906087B0FF221F4094F840328DF8DC
:10ED800009208DF80C308DF80D20002301210DF1A4
:10ED9000090204F510708DF80E3004938DF81530CB
:10EDA0008DF816308DF80F308DF8143000F032FBEE
:10EDB00095F80C31D907F6B20FD59DF80930802BA4
:10EDC0000BD195F8003103F07F0385F8003195F8F9
:10EDD0000C3103F0DF0385F80C317A0711D5BA4BFB
:10EDE000042093F8A41093F8A02083F8800006ABC9
:10EDF00042EA012223F80E2D03A91220049300F009
:10EE00006DFBFB074BD5B04DB0480123BF2685F8FD
:10EE1000803085F8886095F89430002743F002032D
:10EE200085F894304FF4107285F89870FF2185F8BA
:10EE3000007101F03FFB4FF480623946D4F8440280
:10EE400001F038FBD4F8443203F50073C4F84832BB
:10EE50009F4BFF221A7095F8943003F0FD0385F85C
:10EE6000943095F80C3143F0400385F80C319F2322
:10EE700085F88C6085F8843095F8943003F0DF03D2
:10EE800085F8943003A9102000F028FB95F8943001
:10EE900003F0DF0385F8943007B0BDE8F08F3D073D
:10EEA00040F19380884B082283F880203309C6F311
:10EEB000C000062B8DF80D308DF80F0000F2F480A5
:10EEC000C6F3800202EB830208B10232D2B2D4F858
:10EED000446206EBC201C2F34705D1F804E0498859
:10EEE000ADF81510122101FB0541CDF810E091F8A5
:10EEF0000FC08CF0010C81F80FC016F8321082F0B0
:10EF0000010A5FFA8AFAC1F380110FFA8AF881F0D8
:10EF10000101890106EBC80906F83810002800F045
:10EF2000D980DFF8ACB19BB99BF8002082B9FF22F1
:10EF300019468BF8002003A81A460193FFF706FD37
:10EF4000019B06F838301A46194603A8FFF7DCFD86
:10EF50009BF80030012B04D09DF80D30002B00F001
:10EF6000AD80122101FB0541BDF815008B894A894E
:10EF700003449BB293428B8109D3B1F800E0C0B245
:10EF8000864540F09380897B012940F08F801221D3
:10EF900001FB0544D4F8061020881944D31A834293
:10EFA000D8BF98B2A9F80200C9F8041016F83A3090
:10EFB00003F0400363F0770306F83830424A92F8D2
:10EFC000943003F0DF0382F89430B80717D53E4C35
:10EFD000022384F8803094F8883094F88C2003A9B8
:10EFE000134016208DF8143000F078FABF2384F80F
:10EFF000883094F8943003F0DF0384F89430F906F5
:10F000001CD5314C202384F88030102384F88030C4
:10F0100003A9142000F062FA94F80C3143F02003A5
:10F0200084F80C3194F8003143F0800384F8003107
:10F0300094F8843043F0200384F88430BA060DD568
:10F04000214C202384F8803003A9132000F046FAD5
:10F0500094F8843003F0DF0384F884303B067FF5B6
:10F060001BAF0DF10A02FF23102103A88DF80D300C
:10F0700000F0D0F99DF80A30134C012B04BF8DF835
:10F080000F3000224FF0800308BF8DF80D2003A938
:10F0900084F88030172000F021FA94F8943003F0BF
:10F0A000DF0384F89430F7E6FF2210E7122202FB18
:10F0B0000544D4F806200492ADF8153003A99DF854
:10F0C0000D0000F00BFA79E7002007407890FF1F51
:10F0D0005680FF1F6BB916F832202F4902F03C0210
:10F0E000342A35D101238DF80E309EF80030DB092B
:10F0F0000B70122101FB05414FF6FF734A899A42BA
:10F10000DCD0BDF815E08B8973449BB28B810988F4
:10F110008E4501D19A420CD88AB3B2FBF1F001FBC3
:10F12000102080B258BB122000FB0540807B0128D4
:10F1300025D1D21A8A42D8BF91B2122202FB0544CD
:10F14000C9B9D4F80230C9F80430A9F802102DE783
:10F150000A78012ACDD1FF200870194603A801932F
:10F16000FFF7F4FB019B06F838301A46194603A84E
:10F17000FFF7CAFCBDE7D4F806201344E3E71222E8
:10F1800002FB0544D4F80620ADF815304FF0FF33EC
:10F190000492A372E37291E75680FF1F13460A465A
:10F1A000194601F087B900BF30B50329039C0498C4
:10F1B0001DD12BB9164A226004220280002030BDE6
:10F1C00040F209418B420FD1022A4FF000030CD8C4
:10F1D00010490C2505FB0313D9681B6951F822104F
:10F1E00021609B5C0380E9E701230122F0E7072906
:10F1F00001D9CD2030BD074B03EB8102126A22609A
:10F20000002AF6D003EB4103B3F84030EAE700BF31
:10F210005780FF1F640A010001299FBF034B5B5CFD
:10F220001370002088BFCD20704700BFC492FF1F1D
:10F2300001299DBF024B00205A54CD20704700BFCA
:10F24000C492FF1F19B14B1E58425841704701200C
:10F250007047054B1A788A4204D05878431A5842AE
:10F260005841704701207047C492FF1F002070472B
:10F2700000487047B40A010001299FBF044BC1EB4D
:10F28000C101C918002094BF1160CD20704700BF94
:10F290005B80FF1F012930B50ED8084DC1EBC101BD
:10F2A00008231068C45CC818284401330F2B00F8E9
:10F2B000084CF6D1002030BDCD2030BD5B80FF1F53
:10F2C00001299FBF034B03EB41010020116088BF60
:10F2D000CD207047C692FF1F01299FBF034B03EB50
:10F2E00041010020116088BFCD207047CA92FF1FE6
:10F2F00001290AD813681878054B03EB410188707F
:10F3000013685B78CB7000207047CD20704700BF3A
:10F31000C492FF1F01290AD813681878054B03EB24
:10F320004101887113685B78CB7100207047CD2054
:10F33000704700BFC492FF1F084B5A7803F8022B96
:10F34000FF210022D1540132072AFBD1044A0023B5
:10F35000052199540133072BFBD17047CE92FF1F33
:10F36000D792FF1F00BF7047013AD2B2062A10B5EC
:10F370001C4608D8054B5A70FFF7DEFF2146BDE852
:10F380001040FFF7C9B9992010BD00BFCE92FF1FF2
:10F39000024B00225A70FFF731BA00BFCE92FF1F16
:10F3A00037B50F4C257805B9C1B98DF802308DF805
:10F3B00000109DF81830ADF8032069469DF81C2018
:10F3C00000788DF80130FFF737FA9DF800301BB157
:10F3D00010B92378013B237003B030BD9520FBE7C3
:10F3E000CE92FF1F38B50A4B0D461C7859788C42D7
:10F3F0001C4600D14DB929460078FFF7D1FA2DB14E
:10F4000020B923780133237038BD962038BD00BF62
:10F41000CE92FF1F4B1E062B05D8094B19444B7883
:10F42000137000207047CB0607D501F00F010629A5
:10F4300003D8034B19444B7AF2E78220704700BF90
:10F44000CE92FF1F4B1E062B2DE9F041804617463A
:10F4500005D8174B19444A700020BDE8F081CB064F
:10F4600022D501F00F05062D1ED8012A4FEAD1142E
:10F470000F4E06D122462946FFF7C6FA35446F7271
:10F48000EAE7002AFAD173195B7A012BF6D12246FA
:10F490002946FFF789FB002DF0D184F001022946AF
:10F4A0004046FFF781FBE9E78220BDE8F08100BF1D
:10F4B000CE92FF1F00207047062903D9A1F1100347
:10F4C000072B07D8044B53F82130002B0CBFC42066
:10F4D00000207047C4207047DC0A0100102810B5D6
:10F4E0000C4601D1FFF728FF034B53F820300BB136
:10F4F00020469847002010BDDC0A01001FB51446C5
:10F5000002228DF807001A8005210DF10F020DF17E
:10F510000700FFF77FFF034B9DF80F201A80236041
:10F5200004B010BDE092FF1F1FB5144601228DF8F4
:10F5300007001A8004210DF10F020DF10700FFF7FB
:10F5400069FF044B9DF80F201A800020236004B04F
:10F5500010BD00BFE092FF1FF0B5002685B01E80F1
:10F5600049888DF80700ADF80E10FFF76BFE18B351
:10F57000BDF80E20114F04ACB2FA82F252090121FB
:10F580000DF10700FFF75EFF34F8022D0421D2B21F
:10F590000DF10700FFF756FF7B6822460121054663
:10F5A0009DF8070098477B689DF8070032460221C6
:10F5B0009847284605B0F0BD0425FAE7E092FF1F02
:10F5C00073B502AC002504F8010D0E461D8004221F
:10F5D00001212046FFF736FF7288024B28461A7237
:10F5E00002B070BDE092FF1F13B54C8889888DE88A
:10F5F0000C000B46E2B2210AFFF7D6FD02B010BDA7
:10F600002DE9F04186B017461E4606AA002388461B
:10F61000059303238DF80F0002F8083D01210DF139
:10F620000F00FFF7F7FE98F80050274C15F0030580
:10F6300028D10DF1110206210DF10F00FFF7EAFEAE
:10F640009DF811309DF80F0003F0030323800DF1A6
:10F650001203019305AB00932A462B460221FFF7C4
:10F66000A3FD059BDB7913F0400F238814BF43F003
:10F67000010323F001032380022333803C6006B0A2
:10F68000BDE8F081012D08D19DF81030012B02D189
:10F6900098F80430ABB90023EDE7022DEED198F8CD
:10F6A000041041F010010DF11202C9B20DF10F006A
:10F6B000FFF7B0FE9DF8123003F001032380358080
:10F6C000DCE7CD20DAE700BFE092FF1F7FB5002224
:10F6D0001A800B784E788DF8070013F003030D465F
:10F6E000C6F3400634D1FEB14B88013B9BB2012BDF
:10F6F00052D80DF10F0206210DF10700FFF78AFE27
:10F70000044670B9AB7801229A409DF80F301A4335
:10F71000D2B206210DF107008DF80F20FFF792FEFF
:10F720000446204604B070BD4E88012E34D10DF140
:10F730000F0206210DF10700FFF76CFE04460028BA
:10F74000EFD1AA7896409DF80F2022EA0602E0E762
:10F75000022B21D109798DF80F10324641F01001AA
:10F760000DF10700FFF76EFE6B78002E14BF072126
:10F770000821012B044607D19DF80F00C10900F0B4
:10F780000F00FFF7ADF90821044B9DF807005B68F7
:10F790000DF10F029847C4E7CD24C2E7E092FF1FA6
:10F7A00010B500241C800B7803F00303012B05D156
:10F7B0008A780979FFF73CFD204610BD042010BD72
:10F7C00038B515460A7802F00302012A07D1054C24
:10F7D0001A8009792246FFF71FFD2C6038BD0420EE
:10F7E00038BD00BFE092FF1F13B5CD298DF807008B
:10F7F00007D1012290210DF10700FFF723FE02B08F
:10F8000010BD0D491C88088A1268844288BF188080
:10F810000C461B889DF807000021FEF74DFF94F968
:10F820000A30002BEBDA00231A4619460DF10700C7
:10F83000FFF76AF9E3E700BFE092FF1F73B50546E3
:10F8400000266A4601218DF800600196FFF7E2FD6F
:10F85000AA78434C012A52D168680368C4F80A3078
:10F860004368A07AC4F80E3004F10A0110F0600F6A
:10F870001ED1E27A3B4B53F82240002C3DD09DF83C
:10F880000000022839D802EB42021344034493F8E3
:10F890003430012B31D10DF1020301AA2878A047A1
:10F8A0000DF1020301AA01462878FFF79DFF13E03E
:10F8B000238AADF80230202B17D87BB102060DD475
:10F8C0000A68C4F812204A68C4F81620314604F1C8
:10F8D0001A022846FFF718F902B070BDE46B64B154
:10F8E0000DF1020301AA2049D8E702A82B7800F8FD
:10F8F000073D9021FFF7A6FDEEE7CD20D0E79DF86C
:10F900000030042B10D12B78217A02AD05F8063D8A
:10F910002846FFF7D1F9012211462846FFF792FD4C
:10F92000227A03212846E5E794F90A30002BD3DB3D
:10F93000EB78002BD0D1E66B86B1B5F8093028788A
:10F940000833ADF8023004F112010DF1020301AAEF
:10F95000B04701460DF1020301AAA5E7CD21F9E761
:10F96000E092FF1F3C0B0100EA92FF1F034B59601E
:10F97000DA630021024AFFF79DBD00BFE092FF1F3E
:10F980003DF8000007B502AB054A03F8010D002160
:10F9900018465160D163FFF78FFD03B05DF804FB9B
:10F9A000E092FF1F00207047354B41F248015A5842
:10F9B00022F00F0242F002025A5041F204015A585A
:10F9C00042F480225A5041F234015A5842F48022C3
:10F9D0005A5003F52C33602193F8942042F0020230
:10F9E00083F89420C02283F80021FF221A7483F840
:10F9F000802083F8882083F88420002283F88C20DC
:10FA000083F80C111F491A75080A00F0FE0083F8EC
:10FA1000982083F8C02083F8C42083F8C82083F896
:10FA2000CC2083F8D02083F8D42083F8D82083F822
:10FA3000DC2083F8E02083F8E42083F8E82083F8D2
:10FA4000EC2083F8F02083F8F42083F8F82083F882
:10FA5000FC2083F89C00C1F30740090E83F8B00036
:10FA600083F8B41083F8AC201A7783F8082193F850
:10FA7000942002F0D40242F0010283F894207047EF
:10FA800000700440009CFF1F024B4FF400125A60AC
:10FA9000704700BF00E100E0034B4FF40012C3F8D1
:10FAA00084215A60704700BF00E100E008B5FEF70E
:10FAB00082F910B9FFF7F0FF08BD1B2008BD00BF99
:10FAC000034B4AF202629A814BF280429A8170475C
:10FAD0000020054081F0004102E000BF83F00043B8
:10FAE00030B54FEA41044FEA430594EA050F08BFD9
:10FAF00090EA020F1FBF54EA000C55EA020C7FEA9D
:10FB0000645C7FEA655C00F0E2804FEA5454D4EB19
:10FB10005555B8BF6D420CDD2C4480EA020281EAE3
:10FB2000030382EA000083EA010180EA020281EA1B
:10FB30000303362D88BF30BD11F0004F4FEA01316D
:10FB40004FF4801C4CEA113102D0404261EB41017C
:10FB500013F0004F4FEA03334CEA133302D0524202
:10FB600063EB430394EA050F00F0A780A4F10104BE
:10FB7000D5F1200E0DDB02FA0EFC22FA05F28018F8
:10FB800041F1000103FA0EF2801843FA05F35941DE
:10FB90000EE0A5F120050EF1200E012A03FA0EFC5D
:10FBA00028BF4CF0020C43FA05F3C01851EBE37187
:10FBB00001F0004507D54FF0000EDCF1000C7EEBA4
:10FBC00000006EEB0101B1F5801F1BD3B1F5001FE2
:10FBD0000CD349085FEA30004FEA3C0C04F1010401
:10FBE0004FEA445212F5800F80F09A80BCF1004F2A
:10FBF00008BF5FEA500C50F1000041EB045141EAAC
:10FC0000050130BD5FEA4C0C404141EB010111F4AC
:10FC1000801FA4F10104E9D191F0000F04BF014657
:10FC20000020B1FA81F308BF2033A3F10B03B3F135
:10FC300020020CDA0C3208DD02F1140CC2F10C02C5
:10FC400001FA0CF021FA02F10CE002F11402D8BF23
:10FC5000C2F1200C01FA02F120FA0CFCDCBF41EAEF
:10FC60000C019040E41AA2BF01EB0451294330BDBE
:10FC70006FEA04041F3C1CDA0C340EDC04F114049B
:10FC8000C4F1200220FA04F001FA02F340EA030072
:10FC900021FA04F345EA030130BDC4F10C04C4F1B8
:10FCA000200220FA02F001FA04F340EA0300294698
:10FCB00030BD21FA04F0294630BD94F0000F83F4E2
:10FCC000801306BF81F480110134013D4EE77FEAC5
:10FCD000645C18BF7FEA655C29D094EA050F08BF11
:10FCE00090EA020F05D054EA000C04BF19461046F2
:10FCF00030BD91EA030F1EBF0021002030BD5FEA36
:10FD0000545C05D14000494128BF41F0004130BD5D
:10FD100014F580043CBF01F5801130BD01F00045B1
:10FD200045F0FE4141F470014FF0000030BD7FEA24
:10FD3000645C1ABF194610467FEA655C1CBF0B461F
:10FD4000024650EA013406BF52EA033591EA030F36
:10FD500041F4002130BD00BF90F0000F04BF00212E
:10FD6000704730B54FF4806404F132044FF0000561
:10FD70004FF0000150E700BF90F0000F04BF0021DA
:10FD8000704730B54FF4806404F1320410F0004540
:10FD900048BF40424FF000013EE700BF42004FEA3B
:10FDA000E2014FEA31014FEA02701FBF12F07F43B8
:10FDB00093F07F4F81F06051704792F0000F14BFB5
:10FDC00093F07F4F704730B54FF4607401F00045F9
:10FDD00021F0004120E700BF50EA010208BF704750
:10FDE00030B54FF000050AE050EA010208BF704745
:10FDF00030B511F0004502D5404261EB41014FF4AE
:10FE0000806404F132045FEA915C3FF4DCAE4FF0B1
:10FE100003025FEADC0C18BF03325FEADC0C18BF98
:10FE2000033202EBDC02C2F1200300FA03FC20FAE9
:10FE300002F001FA03FE40EA0E0021FA02F1144436
:10FE4000C1E600BF70B54FF0FF0C4CF4E06C1CEA4B
:10FE500011541DBF1CEA135594EA0C0F95EA0C0FC0
:10FE600000F0DEF82C4481EA030621EA4C5123EA33
:10FE70004C5350EA013518BF52EA033541F4801162
:10FE800043F4801338D0A0FB02CE4FF00005E1FB15
:10FE900002E506F00042E0FB03E54FF00006E1FB5F
:10FEA00003569CF0000F18BF4EF0010EA4F1FF04A2
:10FEB000B6F5007F64F5407404D25FEA4E0E6D41E2
:10FEC00046EB060642EAC62141EA55514FEAC520F3
:10FED00040EA5E504FEACE2EB4F1FD0C88BFBCF56F
:10FEE000E06F1ED8BEF1004F08BF5FEA500E50F120
:10FEF000000041EB045170BD06F0004646EA0101E6
:10FF000040EA020081EA0301B4EB5C04C2BFD4EB17
:10FF10000C0541EA045170BD41F480114FF0000E10
:10FF2000013C00F3AB8014F1360FDEBF002001F07E
:10FF3000004170BDC4F10004203C35DA0C341BDCF8
:10FF400004F11404C4F1200500FA05F320FA04F0CA
:10FF500001FA05F240EA020001F0004221F00041FE
:10FF600010EBD37021FA04F642EB06015EEA430E71
:10FF700008BF20EAD37070BDC4F10C04C4F12005A1
:10FF800000FA04F320FA05F001FA04F240EA020054
:10FF900001F0004110EBD37041F100015EEA430E25
:10FFA00008BF20EAD37070BDC4F1200500FA05F245
:10FFB0004EEA020E20FA04F301FA05F243EA0203C4
:10FFC00021FA04F001F0004121FA04F220EA0200D3
:10FFD00000EBD3705EEA430E08BF20EAD37070BD19
:10FFE00094F0000F0FD101F00046400041EB0101F9
:10FFF00011F4801F08BF013CF7D041EA060195F0DB
:020000021000EC
:10000000000F18BF704703F00046520043EB030394
:1000100013F4801F08BF013DF7D043EA0603704781
:1000200094EA0C0F0CEA135518BF95EA0C0F0CD08C
:1000300050EA410618BF52EA4306D1D181EA0301D2
:1000400001F000414FF0000070BD50EA410606BFCC
:100050001046194652EA430619D094EA0C0F02D111
:1000600050EA013613D195EA0C0F05D152EA033656
:100070001CBF104619460AD181EA030101F0004174
:1000800041F0FE4141F470014FF0000070BD41F0BD
:10009000FE4141F4780170BD70B54FF0FF0C4CF497
:1000A000E06C1CEA11541DBF1CEA135594EA0C0FB6
:1000B00095EA0C0F00F0A7F8A4EB050481EA030E03
:1000C00052EA03354FEA013100F088804FEA0333EA
:1000D0004FF0805545EA131343EA12634FEA0222B8
:1000E00045EA111545EA10654FEA00260EF0004179
:1000F0009D4208BF964244F1FD0404F5407402D2CB
:100100005B084FEA3202B61A65EB03055B084FEA5B
:1001100032024FF480104FF4002CB6EB020E75EB58
:10012000030E22BFB61A754640EA0C005B084FEA80
:100130003202B6EB020E75EB030E22BFB61A7546FD
:1001400040EA5C005B084FEA3202B6EB020E75EB48
:10015000030E22BFB61A754640EA9C005B084FEAC0
:100160003202B6EB020E75EB030E22BFB61A7546CD
:1001700040EADC0055EA060E18D04FEA051545EABC
:1001800016754FEA06164FEAC30343EA52734FEA65
:10019000C2025FEA1C1CC0D111F4801F0BD141EADE
:1001A00000014FF000004FF0004CB6E711F4801F43
:1001B00004BF01430020B4F1FD0C88BFBCF5E06F23
:1001C0003FF6AFAEB5EB030C04BFB6EB020C5FEA33
:1001D000500C50F1000041EB045170BD0EF0004E88
:1001E0004EEA113114EB5C04C2BFD4EB0C0541EABA
:1001F000045170BD41F480114FF0000E013C90E6B7
:1002000045EA060E8DE60CEA135594EA0C0F08BF7A
:1002100095EA0C0F3FF43BAF94EA0C0F0AD150EA79
:1002200001347FF434AF95EA0C0F7FF425AF10460C
:1002300019462CE795EA0C0F06D152EA03353FF434
:10024000FDAE1046194622E750EA410618BF52EAB1
:1002500043067FF4C5AE50EA41047FF40DAF52EA85
:1002600043057FF4EBAE12E74FF0FF3C06E000BF22
:100270004FF0010C02E000BF4FF0010C4DF804CD2F
:100280004FEA410C7FEA6C5C4FEA430C18BF7FEAEF
:100290006C5C1BD001B050EA410C0CBF52EA430C1D
:1002A00091EA030F02BF90EA020F0020704710F19D
:1002B000000F91EA030F58BF994208BF90422CBF2C
:1002C000D8176FEAE37040F0010070474FEA410C25
:1002D0007FEA6C5C02D150EA013C07D14FEA430C43
:1002E0007FEA6C5CD6D152EA033CD3D05DF8040BB4
:1002F000704700BF8446104662468C4619466346E6
:1003000000E000BF01B5FFF7B7FF002848BF10F1BC
:10031000000F01BD4DF808EDFFF7F4FF0CBF012001
:1003200000205DF808FB00BF4DF808EDFFF7EAFF7D
:1003300034BF012000205DF808FB00BF4DF808ED38
:10034000FFF7E0FF94BF012000205DF808FB00BF2D
:100350004DF808EDFFF7CEFF94BF012000205DF8B7
:1003600008FB00BF4DF808EDFFF7C4FF34BF0120C4
:1003700000205DF808FB00BF4FEA410212F50012B1
:1003800015D211D56FF47873B3EB625212D94FEADC
:10039000C12343F0004343EA505311F0004F23FAC6
:1003A00002F018BF404270474FF00000704750EA1B
:1003B000013005D111F0004008BF6FF000407047D8
:1003C0004FF00000704700BFFDF7BDFB002103E0C8
:1003D0000A4B5B584350043109480A4B42189A4271
:1003E000F6D3094A02E0002313600432074B9A4215
:1003F000F9D300F00DF8804770470000C80B0100EA
:100400000880FF1F6C85FF1F0086FF1F24A0FF1FB1
:10041000254C08B5F8F735F8F8F79CF8F8F702FA24
:10042000F8F714FAF8F71EF9F8F7F4FBFCF712FDE9
:10043000FCF7FAFAF8F75AFDF8F7A6FA2078F8F779
:1004400021F9E078F8F78EF9F8F747FB28B1F8F7CB
:1004500044FB6070F8F741FBA060F8F7B7FB218917
:100460006079228AFCF73AFBFDF710FAFCF788FD69
:100470000E4B4FF400725A60FBF718F9FBF7E0FDE2
:100480000B4B04225A60FBF737FAFBF717FEFBF71A
:10049000D8FDF8F756FBF8F789FB0028F3D0FDF7F5
:1004A000F5F9FBF703F9EEE70C80FF1F80F00F4032
:1004B00000F00F4070B4860746D0541E002A41D089
:1004C000CAB2034602E014F1FF343BD303F8012B18
:1004D0009D07F8D1032C2ED9CDB245EA05250F2C66
:1004E00045EA054519D903F110022646103E0F2EA4
:1004F00042F8105C42F80C5C42F8085C42F8045C7C
:1005000002F11002F2D8A4F1100222F00F0204F05E
:100510000F041032032C13440DD91E462246043A10
:10052000032A46F8045BFAD8221F22F003020432A1
:10053000134404F003042CB1C9B21C4403F8011B9A
:100540009C42FBD170BC704714460346C2E700BF13
:100550002DE9F84355EC104BC5F30A52A2F2FF33D4
:10056000132B064612DC002B41DB244A42FA03F32C
:1005700005EA030252EA040017D105F000430246DF
:1005800086ED000B43EC102BBDE8F883332B1CDC0D
:10059000A2F213424FF0FF3323FA02F214EA0207E9
:1005A0001CD0A94624EA020803E04FF0000825EA1F
:1005B000030942464B4620462946C6E90023FFF779
:1005C0008DFA41EC100BBDE8F883002205F00043E2
:1005D00086ED000B43EC102BBDE8F88305F00043DB
:1005E0003A4686ED000B43EC102BBDE8F883002261
:1005F00005F00043C6E90023BDE8F883FFFF0F00C4
:10060000024B13B1024800F005B87047000000002B
:1006100021060100002301461A46184600F01EB8C4
:1006200038B50A4C0A4D641BA4100AD004F180436B
:10063000013B05EB8305013C55F804399847002C34
:10064000F9D1BDE8384000F0B3BA00BFC80B0100D3
:10065000C40B0100704700BF704700BF2DE9F8438D
:100660002C4D0646286898460F469146FFF7F2FF44
:10067000294B1C68D4F84831002B3ED05A681F2AF9
:100680001CDC02F1010E76B103EB82010124C1F8FA
:100690008890D3F8880194402043022EC3F8880143
:1006A000C1F8088123D00232C3F804E0286843F877
:1006B0002270FFF7D1FF0020BDE8F883174B0BB382
:1006C0004FF4C870AFF300800346D8B1D4F8482186
:1006D0000260002141600A46C4F848014FF0010E53
:1006E000C0F88811C0F88C11002EDCD0CCE7D3F80C
:1006F0008C110C43C3F88C41D5E704F5A673C4F8FC
:100700004831BBE72868FFF7A7FF4FF0FF30BDE88F
:10071000F88300BF6885FF1FA00B010000000000E8
:1007200051EC100B2DE9F843C1F30A59A9F2FF353A
:10073000132D0C4610EE106A884610EE107A22DC5B
:10074000002D52DB3E4B43FA05F901EA090303434E
:100750001ED039A3D3E90023FFF7C2F900220023FA
:10076000FFF700FE48B1002C04DD4FF4801343FA7C
:1007700005F5A84428EA0904002723463A4643EC35
:10078000102BBDE8F883332D06DDB5F5806F3FD023
:1007900041EC100BBDE8F883A9F213494FF0FF3389
:1007A00023FA09F910EA090FF2D023A3D3E90023B1
:1007B000FFF796F900220023FFF7D4FD0028DCD0D4
:1007C000002C09DD142D32D00127C5F1340507FABC
:1007D00005F5AE1928BFB844444626EA0907234662
:1007E0003A4643EC102BBDE8F88313A3D3E900236A
:1007F000FFF776F900220023FFF7B4FD0028BCD0F4
:10080000002C10DB54EA06070BD000270D4CB4E790
:1008100010EE102A0B46FFF763F941EC100BBDE810
:10082000F8833C46A9E700274FF00044A5E704F110
:100830000108D1E7AFF300809C7500883CE4377E67
:10084000FFFF0F000000F03F51EC100BC1F30A5303
:100850002DE9F041A3F2FF35132D0C460F4610EEA3
:10086000106A1DDC002D43DB3D4B43FA05F801EA1D
:100870000803034319D038A3D3E90023FFF730F965
:1008800000220023FFF76EFD20B1002C49DB27EA90
:10089000080400262346324643EC102BBDE8F081C5
:1008A000332D06DDB5F5806F32D041EC100BBDE87D
:1008B000F081A3F213434FF0FF3828FA03F810EA4F
:1008C000080FF2D024A3D3E90023FFF709F900228F
:1008D0000023FFF747FD0028DCD0002C27DB3C4637
:1008E00026EA08062346324643EC102BBDE8F08189
:1008F00019A3D3E90023FFF7F3F800220023FFF741
:1009000031FD0028C6D0002C1CDB00263446C1E790
:1009100010EE102A0B46FFF7E3F841EC100BBDE890
:10092000F0814FF4801343FA05F52F44AFE7142DFF
:1009300010D00123C5F1340503FA05F5AE1928BF1F
:10094000FF18CCE724F00042064B324318BF1C4688
:1009500000269FE70137C2E79C7500883CE4377E9C
:10096000FFFF0F000000F0BF8025000040380000AE
:10097000004B0000807000000096000000E10000C5
:10098000002C010000C201000084030090D003008D
:1009900020A1070040420F0050C300008813000050
:1009A000018008080000000000000000C8000000EE
:1009B0000100C800008000000000000000000000EE
:1009C0000000000000000000000000000000000027
:1009D0000000000000000000010002000400080008
:1009E00010002000010101000100000000000000D3
:1009F00000000000000001000000000000000000F6
:100A000000000000010101000000000000000000E3
:100A100000010000000000000101010001010001CF
:100A200001000000000000000000000000000000C5
:100A300000000000000000000000000000000000B6
:100A400000000000000000000000000000000101A4
:100A50000100000100010001000000000000000092
:100A6000000000005780FF1F040000000904000080
:100A7000C80A0100D80A01000000000000000000C0
:100A800000000000000000002E81FF1FEB80FF1F10
:100A90000000000000000000000000000000000056
:100AA00000000000000012004300000000000000F1
:100AB0000000000003010201100002020010000308
:100AC00003011000000100005780FF1FB180FF1FCD
:100AD0008B80FF1F6980FF1F043A26223DF800002B
:100AE00039E10000D1E1000041DF000065F30000C2
:100AF00065F3000065F3000065F3000065F3000096
:100B000065F3000065F3000065F3000065F3000085
:100B100065F3000065F3000065F30000C3E4000026
:100B200059E40000B9E4000085E4000059E4000045
:100B300065F3000045E4000031E5000001F6000027
:100B4000CDF6000000000000CDF60000000000001F
:100B5000C1F50000E9F500000000000029F50000E3
:100B600059F50000C1F70000A1F70000FDF40000F6
:100B7000010100010100000000010100000000006F
:100B8000010101010100000001010001010001005B
:100B9000000100000100003332313456313037009B
:100BA0004081FF1FF8B500BFF8BC08BC9E467047E7
:0C0BB000F8B500BFF8BC08BC9E467047BA
:080BBC00010601003584000070
:040BC4001184000098
:100BC800970B01000001020000080000010000006E
:100BD800020000000000000000000000000000000B
:100BE80000000000000000000000000000000000FD
:100BF80000000000000000000000000000000000ED
:100C080000000000A1200000000002000000FF0416
:100C180003090400C20100000008000000000000F1
:100C280000220342004100440020005300540052B7
:100C38000049004E004700200049004E004400458E
:100C480000580026035300740065007000700065AA
:100C580000720020004D006F0074006F00720020C9
:100C68000044006500760020003A03540052004911
:100C7800004E0041004D004900430020004D006F28
:100C880000740069006F006E00200043006F006E62
:100C980000740072006F006C00200020002000200B
:100CA80000200009024300020100C03209040000CC
:100CB80001020200000524001001052401010104BD
:100CC80024020605240600010705830310000A090B
:100CD800040100020A000000070581021000000755
:100CE80005020210000012010002020000103C2A56
:100CF8000001020001020001000000002C84FF1F17
:100D08009484FF1FFC84FF1F000000000000000007
:100D180000000000000000000000000000000000CB
:100D280000000000000000000000000000000000BB
:100D380000000000000000000000000000000000AB
:100D4800000000000000000000000000000000009B
:100D5800000000000000000000000000000000008B
:100D6800000000000000000000000000000000007B
:100D7800000000000000000000000000000000006B
:100D8800000000000000000000000000000000005B
:100D9800000000000000000000000000000000004B
:100DA80001000000000000000E33CDAB34126DE6E8
:100DB800ECDE05000B000000000000000000000051
:100DC800000000000000000000000000000000001B
:100DD800000000000000000000000000000000000B
:100DE80000000000000000000000000000000000FB
:100DF80000000000000000000000000000000000EB
:0411280000A0FF1F05
:10112C00C80B01000880FF1F6405000000000000D0
:08113C000000000000000000AB
:020000020000FC
:020000041FFFDC
:04800000000000007C
:04000003100003C91D
:00000001FF
